:020000040002F8
:10600000E0510020C1630200C9630200CB630200BB
:10601000CD630200CF630200D163020000000000E4
:10602000000000000000000000000000D363020038
:10603000D563020000000000D7630200D9630200AC
:1060400091670200DB630200F1690200DB6302007A
:10605000DB630200DB63020079650200DB630200A0
:10606000DB630200DB630200DB630200DB63020030
:10607000DB630200DB630200DB630200DB63020020
:10608000DB630200E9670200DB630200DB630200FE
:106090000D680200DB63020011680200DB6302008E
:1060A000DB630200DB630200DB630200DB630200F0
:1060B000DB630200DB630200000000000000000060
:1060C000DB630200DB630200DB630200DB630200D0
:1060D000DB630200DB630200DB630200DB630200C0
:1060E000DB630200DB630200DB63020000000000F0
:1060F00000000000DB63020000000000DB63020020
:10610000000000000000000000000000000000008F
:10611000000000000000000000000000000000007F
:10612000000000000000000000000000000000006F
:10613000000000000000000000000000000000005F
:10614000000000000000000000000000000000004F
:10615000000000000000000000000000000000003F
:10616000000000000000000000000000000000002F
:10617000000000000000000000000000000000001F
:10618000000000000000000000000000000000000F
:1061900000000000000000000000000000000000FF
:1061A00000000000000000000000000000000000EF
:1061B00000000000000000000000000000000000DF
:1061C00000000000000000000000000000000000CF
:1061D00000000000000000000000000000000000BF
:1061E00000000000000000000000000000000000AF
:1061F000000000000000000000000000000000009F
:10620000DFF80CD000F07AF900480047A1A30200A3
:10621000E051002030B450E8012F93B2C4892344E8
:106220008489A34228BF1B1B0489A34202BFBFF37A
:106230002F8F002007E0C3EA020340E80134002C5E
:10624000E9D14FF001000A6030BC704750E8012FDF
:10625000C2EA024240E801210029F7D1704730B478
:1062600050E8022F1FFAA2F3C488A34202BFBFF373
:106270002F8F00200DE0C48923448489A34228BFC6
:106280001B1BC2EA034340E80234002CE8D14FF064
:1062900001000A6030BC704750E8022FC2EA224277
:1062A00040E802210029F7D17047034653E8022F46
:1062B000D988B2EB324F4FF0000017BF92B241EADB
:1062C000014142EA014104E05A68B2EB324F08BF93
:1062D000012043E80212002AE8D1704730B4044696
:1062E00054E8000F0D4644E80053002BF8D1156028
:1062F00030BC704730B4044654E8000F40EA010552
:1063000044E80053002BF7D1156030BC704730B41F
:10631000044654E8000F00EA010544E80053002B4E
:10632000F7D1156030BC704730B4044654E8000F14
:1063300080EA010544E80053002BF7D1156030BC1A
:10634000704730B4044654E8000F00EB010544E800
:106350000053002BF7D1156030BC704730B40446B1
:1063600054E8000FA0EB010544E80053002BF7D1DF
:10637000156030BC704770B404464FF0000054E81C
:10638000006F0D68AE4207BF44E80023012044E8D7
:1063900000630E60002B1CBF0020F0E770BC70474C
:1063A00030B4044654E8000F88422CBF451A054615
:1063B00044E80053002BF5D1156030BC7047000055
:1063C0000648804706480047FEE7FEE7FEE7FEE78F
:1063D000FEE7FEE7FEE7FEE7FEE7FEE715680200E0
:1063E000016202002DE9F05F0546002092469B46BF
:1063F00088460646814640241BE0284641464746DB
:10640000224600F06BF853465A46C01A914110D309
:1064100011461846224600F016F82D1A67EB0108BF
:106420004F4622460120002100F00DF817EB00092D
:106430004E41201EA4F10104DFDC484631462A46C5
:106440004346BDE8F09F202A04DB203A00FA02F11F
:10645000002070479140C2F1200320FA03F3194352
:1064600090407047004870479800030040EA0103DD
:106470009B0703D009E008C9121F08C0042AFAD2FA
:1064800003E011F8013B00F8013B521EF9D27047BE
:10649000D2B201E000F8012B491EFBD27047002266
:1064A000F6E710B513460A4604461946FFF7F0FF13
:1064B000204610BD421C10F8011B0029FBD1801A98
:1064C000704730B504460020034600E05B1C934251
:1064D00003D2E05CCD5C401BF8D030BD202A04DB49
:1064E000203A21FA02F00021704721FA02F3D0404D
:1064F000C2F120029140084319467047064C074DEF
:1065000006E0E06840F0010394E807009847103483
:10651000AC42F6D3FFF778FEDC080300FC0803006A
:1065200070B58C1810F8015B15F0070301D110F855
:10653000013B2A1106D110F8012B03E010F8016B82
:1065400001F8016B5B1EF9D12B0705D40023521E05
:106550000DD401F8013BFAE710F8013BCB1A921C6D
:1065600003E013F8015B01F8015B521EF9D5A1426B
:10657000D8D3002070BD00002DE9F04F00268DB06B
:10658000DFF8A081B14604964FF4807501243746A8
:106590000596284605F05AF938B1D8F80403204288
:1065A00003D0284605F048F926432D1D64007F1CC2
:1065B000ADB2082FEDD34FF4BE74204605F046F976
:1065C00048B1204605F038F946F0004604AA0221F9
:1065D000002005F01BF9544C16F0FF0F15D00127D1
:1065E000002537420DD008EB8501D1F81005D1F810
:1065F0001015C0F3052054F82520C1F3014102B164
:1066000090477F006D1C082DEBD3002E7EDA002012
:10661000CDF82890411E0DF1100B07AACDF82C9053
:1066200042F82010401C91460228F9D300252E463E
:10663000A11911F8607F91F9000027F0C008401CF3
:1066400040D007A9404604F0FAF940B34FEA971A40
:10665000404602F02FF854F820701FB1BAF1030F32
:1066600003D006E0BAF1030F2CD10AA9404604F08A
:10667000EEF902A8CDF8088005F06CF8029900EB5D
:106680008100D0F8000704A9C0F301400290404601
:1066900004F0D5F90028029802D0022802D011E0B7
:1066A00003280FD1BAF1030F08D10298022833D082
:1066B0000221404605F028F86D1CEDB217B1514695
:1066C0004046B847761C042EB2D3002D21D001AA33
:1066D0000221002005F09AF800205A460DF104012D
:1066E00052F8206051F82030B34217D000200AAE93
:1066F0004FEA090351F8207042F8207056F82070D4
:1067000043F82070401C0228F4D300E001E0002D83
:106710008CD10DB0BDE8F08F0321CAE7401C0228E0
:10672000DED3F6E7006000401829002000F01F02C9
:10673000012191404009800000F1E020C0F8801262
:10674000704700F01F02012191404009800000F1D4
:10675000E020C0F80011704700F01F0201219140B5
:106760004009800000F1E020C0F80012704749079E
:10677000090E002806DA00F00F0000F1E02080F892
:10678000141D704700F1E02080F8001470470000ED
:1067900070B54FF48076304604F090FA114CB50590
:1067A00060B1304604F091FA0120C5F80803607921
:1067B00020B9012060712168002088474FF482765B
:1067C000304604F07BFA00280AD0304604F07DFA07
:1067D0000220C5F808032168BDE870400120084781
:1067E00070BD0000B822002007480021C0F8401109
:1067F000C0F84411C0F84811C0F84C11C0F800119D
:10680000C0F8041108F098BC0010014008F0E2BB89
:1068100005F0C6BD30B54FF0805000228300D0F89F
:106820003011C3F80C21C3F81021624B1A60624B7F
:106830001B68624C2360604B1B1D1B68241D23607A
:106840005D4B08331B68241D23605B4B0C331B68B6
:10685000241D2360584B10331B68241D2360564BA6
:1068600014331B68241D2360534B18331B68534C8F
:1068700020342360504B1C331B68241D23604E4B77
:1068800020331B68241D23604B4B24331B68241DBD
:106890002360494B28331B68241D2360464B2C334F
:1068A0001B68241D2360444B30331B68434C403429
:1068B0002360414B34331B68241D23603E4B383327
:1068C0001B68241D23603C4B3C331B68241D236044
:1068D000394B40331B68241D23600124082902D151
:1068E000D0F8343113B1082904D006E0354B3449CF
:1068F000196005E0D0F8343113B1082904D006E05E
:10690000314BFB21196005E0D0F8343113B108296F
:1069100008D00EE090F858322C48016863F3030168
:10692000016002E0D0F834311BB929494FF40070FE
:10693000086028480168C90702D06FF001010160B2
:106940002548016841F470010160BFF34F8FBFF328
:106950006F8F4FF01021D1F80002002803DBD1F82F
:106960000402002822DA1D4B1C601D480468002C1C
:10697000FCD01224C1F800420568002DFCD0C1F8FB
:10698000044201680029FCD01A6001680029FCD08B
:10699000BFF34F8F10487C380168124A01F4E06160
:1069A00011430160BFF34F8F00BFFDE70F490E4851
:1069B000086030BD380500400404001020C50040C8
:1069C000488103008C56004018F50040E40E00405A
:1069D000409602400004004088ED00E004E50140DC
:1069E00000E401400400FA050090D003DC230020FD
:1069F0000148006800470000C022002002E008C8EB
:106A0000121F08C1002AFAD170477047002001E028
:106A100001C1121F002AFBD170470000012120286C
:106A200003DA81400548014003E0402802DA2038BB
:106A3000814009B10120704700207047FC06FFBD6E
:106A400010B560B159B102780B785208B2EB530F10
:106A500005D10622401C491CFFF733FD08B1002078
:106A600010BD012010BD800701D00020704701201B
:106A70007047C3688B4206D811440069491E8142A1
:106A800001D8012070470020704710B50122022173
:106A9000002001F013FC08B1072810D107220221C1
:106AA000012001F00BFC08B1072808D100210A22BF
:106AB000084601F003FC08B1072800D1002010BDF2
:106AC00010B550B10A480321008801EB004009A12C
:106AD00005F0ACF807F078F903E00321094800F06D
:106AE000A0FC002803D0BDE8104000F0CBB810BDDA
:106AF00024240020457261736520626F6E647321E7
:106B0000000000005424002070B58CB015460E46DD
:106B100000236C46C3F10F01415CE1545B1C102B58
:106B2000F8D30D2104F11000FFF7B9FC0020C0F1EB
:106B30000F02315C2244401C11740328F7D36846CD
:106B400046DF0020C0F10F01214491F820102954A4
:106B5000401C0328F6D30CB070BD022001F0B0BA7F
:106B60000149097900F0F0BD8022002070B50024B1
:106B7000064D06E06868012110F8340005F0FAFCC3
:106B8000641C28788442F5D3002070BDC822002000
:106B9000F8B515460C460646052A01D20720F8BD71
:106BA00005F0E0FD18B905F0A3FD0028F7D1124962
:106BB00000224E600C708D60C1E90422C1E90622FA
:106BC0000E4D0DE006EBC4002968009181788DF828
:106BD000011000780A4A694605F018FD0028DED148
:106BE000641EE4B2EED2BDE8F84004480021054A34
:106BF000001D00F099B80000C822002010FD02001E
:106C00001D970200018B020072B605F0C5F800BFA7
:106C100004F0FCFE0028FBD1104C0121208801EB80
:106C200000400FA105F002F810480068C00700D02E
:106C300000BE2088022101EB00400DA104F0F6FF08
:106C4000BFF34F8F0948E43801680D4A01F4E06151
:106C500011430160BFF34F8F00BFFDE724240020E4
:106C6000466174616C206572726F7200F0ED00E035
:106C700053797374656D207265736574000000004C
:106C80000400FA050EB500210091CDE901106A4615
:106C900044F20100FFF7B8FF0EBD000070B50228F6
:106CA0000DD1084C032508A1208805EB004004F015
:106CB000BDFF208810A105EB004004F0B7FF0120C4
:106CC00070BD000024240020506F776572206D6134
:106CD0006E6167656D656E742077616E7473207484
:106CE0006F20726573657420746F20444655206D63
:106CF0006F64652E00000000506F776572206D6133
:106D00006E6167656D656E7420616C6C6F7765642C
:106D100020746F20726573657420746F204446552B
:106D2000206D6F64652E0000074B9B7823B12AB15C
:106D300020B10068037C1BB1082070470720704712
:106D40004174426100207047F429002070B507F0BB
:106D500065FB104800240B21047044700E4D8170B7
:106D600014206C602C706C70FFF7E0FC072114207D
:106D7000FFF7FDFC1420FFF7E4FC0848046007213E
:106D80001120FFF7F4FC0548001F0068A8600020F0
:106D900070BD0000F4290020E82200200815014001
:106DA0002DE9FC47DFF8789099F8023073B368B3A7
:106DB000052902D20720BDE8FC87436933B3437C31
:106DC000012B25D0002704460025884616468DF85D
:106DD0000050684600F038F801A808F043FCC8B13C
:106DE000012101700F4944600968C0E90218C0E937
:106DF00004769DF8040089F801009DF8000000F079
:106E000047F81420FFF7A8FC2846D4E70820D2E76B
:106E10000F46D8E704259DF8000000F039F8F3E7A5
:106E2000F4290020041501400649897839B130B1B0
:106E3000416921B100210174022108F059B90820EB
:106E400070470000F429002030B5EFF3108172B6CE
:106E50000D4A9468012324B10370002900D162B661
:106E600030BD93604FF0E023D3F88051074C2540AC
:106E70001560C3F88041D3F8844154605A17C3F8B1
:106E8000842100220270E8E7002B0020FC06FFBDF1
:106E90000B498A68002A11D000280FD1EFF3108027
:106EA00072B60B684FF0E022C2F800314B68C2F8AE
:106EB000043100228A60002800D162B670470000C9
:106EC000002B002070B5054608680C46411C04D014
:106ED00004F075FC206804F003FC6068411C02D0DB
:106EE000002104F0EBFB2968A069C1F82405607D4E
:106EF000227D29681043C1F86C05D4E90012286886
:106F0000C0F81425C0F80C15207D012814D1A06804
:106F1000411C02D0002104F0D1FBE068411C04D0E8
:106F200004F04DFCE06804F0DBFBD4E902122868B1
:106F3000C0F80825C0F8101570BD70B50546086882
:106F40000C46411C04D004F044FC206804F0D2FB41
:106F50006068411C02D0002104F0B9FB2968A069D7
:106F6000C1F82405607D217D2A680843C2F86C05BC
:106F7000D4E900122868C0F80C15C0F81425207D4B
:106F8000012814D1A068411C02D0002104F09FFB0D
:106F9000E068411C04D004F01CFCE06804F0AAFB8B
:106FA000D4E902122868C0F80825C0F8101570BD91
:106FB00003F052B92DE9F047074600888EB08046AD
:106FC00002F040FE824604462D4800252A460178FC
:106FD000404600F0D1FB7879400734D501254FF6C3
:106FE000FF7603AB2A460721504606F0CFF8010092
:106FF00004D0404607F00AFC00252BE0B14631469C
:10700000049802F073FD064648450FD00446014639
:10701000404602F001FE4046FFF7A2FD30B940466F
:1070200007F0C6FB4046FFF79BFD48B1224607210B
:10703000504606F021F9010003D0404607F0E6FB78
:1070400000254E4506D0404606F084FA10B1504661
:1070500002F0E4FD02208DF81800ADF81A8078796E
:10706000400701D5012000E002208DF820008DF8B6
:10707000215006A801F004FF0EB0BDE8F087000023
:10708000802200202DE9FC47002517880646158040
:1070900090F82D001446894630B13A4621464846BC
:1070A00000F094FB051E09D1B0784FF00C0A18B31C
:1070B0002088C846001DB84202D95046BDE8FC876A
:1070C000684679DF0028F9D12088032108F80010EC
:1070D00020881921401C80B2208008F800102088E8
:1070E000401C80B2208000EB0801BDF8000008F0D1
:1070F000E7F9218808442080F0780222C8B121886D
:1071000096F9033001F1030C4846BC45D5D84254EA
:1071100021884FF0010C491C89B2218000F801C080
:107120002188491C89B2218009F801302088401C3F
:1071300020807068B8B1218890F9003001F1030C0B
:107140004846BC45B9D8425421880A22491C89B214
:10715000218042542188491C89B2218009F80130DC
:107160002088401C2080308950B1CDE900474B4633
:107170000622022106F1080008F08CFA051E9DD1B6
:10718000308A50B1CDE900474B460722032106F172
:10719000100008F07FFA051E90D1308B50B1CDE978
:1071A00000474B461522142106F1180008F072FA28
:1071B000051E83D1306A30B13B462246494601F074
:1071C00034FB051EDBD1706A30B13B46224649468E
:1071D00003F0F0F9051ED2D196F82C0038B13B46E9
:1071E00022464946304607F0B7FB051EC7D1307826
:1071F00038B13B4622464946304603F061FA051E47
:10720000BDD128465AE718B504460020ADF8000065
:1072100013466A46204600F006F8002802D0BDF862
:107220000000204418BD70B588B182B100241588D3
:1072300003E0065D641C3444A4B2A54203D80619D9
:1072400076789E4201D08C42F3D38C4201D3002049
:1072500070BDA11C1180005D401E80B270BD80F821
:10726000301070472DE9F0410E00044606D02CB1D5
:1072700096F87A000025012803D006E00E20BDE82C
:10728000F08196F89800012821D04FF00108A570F0
:107290002C2206F17801201DFFF7E8F884F8305021
:1072A000D6F8A4006063D6F8A800A0634FF6FF707C
:1072B000A4F8A80004F19400C4F8A400C4F8AA50EB
:1072C000A4F8AE5084F8B050207810B104E0072044
:1072D000D5E7FF2084F8540004F155011F27C4F8B6
:1072E0009410A4F8987004F198023046FFF7CAFE93
:1072F0000028C4D116F13C0F0ED004F17401C4F87B
:107300009C10A4F8A07004F1A00206F13C00FFF765
:10731000B9FE0028B3D103E0C4F89C50A4F8A050F3
:1073200084F85180208BA4F8480084F83C802564C0
:1073300084F8505060696064464604F13C020021C4
:1073400004F1540072DF002899D1267097E710B538
:107350000288102A1BD0112A20D0262A1DD1007A9B
:107360000C46012801D0022817D1A0780521401C25
:10737000B0FBF1F201FB1201204600F052F80028A8
:107380000BD0A16B002908D0BDE810400847C27B94
:10739000012A02D18088A1F8A80010BD0C46002166
:1073A00084F8B2108088B4F8A8108842F5D120790A
:1073B0000028F2D10121DFE710B50C46022801D0E8
:1073C000032810D1607800280DD000206070A178CB
:1073D000204600F026F8002805D0A16B002902D035
:1073E000BDE81040084710BD10B5044690F85400A1
:1073F00074DF012084F8B200002084F8B40084F81F
:1074000050000621204601F041FF002808D1A17854
:10741000204600F006F810B1A16B01B188470020AA
:1074200010BD2DE9F05F044600780F4638B1A77013
:10743000002003F04DFF012620B1667007E108200F
:10744000BDE8F09F0025C4F8AA50A4F8AE5084F817
:10745000B050A07910B1A078012806D0E07968B1C9
:10746000A078012801D0022808D1616B21B184F8ED
:10747000B1600820884701E084F8B15004F1AB0105
:1074800000200A5C0AB1304603E0401C0628F8D30D
:1074900000204FF002084FF0030B012F06D0022FFF
:1074A0000CD0032F0FD0042F15D110E0A17929B1F2
:1074B00094F8241011B908B130460DE0E17911B10A
:1074C00008B1404608E0207A08B1584604E0607AE6
:1074D00008B1042000E02846A070616B41B1032888
:1074E00001D0042804D1607910B194F8B200A0B1A1
:1074F00084F8B35004F13C0018210746FEF7CFFF93
:1075000004F12C0084F83C60814606F05FF958B124
:1075100094F82C0084F8510008E084F8B45084F802
:10752000B36007208847E5E784F8516094F82400A9
:1075300050B1484606F04AF920B194F8280084F882
:10754000520001E084F8526084F85050A27804F1AF
:10755000AA0104F194094FF0060A052A60D2DFE877
:1075600002F078030F223F0084F83160C4F8A45081
:10757000C4E9101584F83C808020A4F8480051E04C
:1075800084F8318094F82420384612B10722027022
:1075900001E080F800B0228A8281C4F8A4504160E2
:1075A000E168B9603EE06069B860208BB88194F80A
:1075B00024003D4610B184F83CA001E084F83C6012
:1075C000204608F02BF840B185F8148004212046AD
:1075D00001F05CFE20BB05211EE084F831B01DE007
:1075E000E069B860208CB88194F824003D4610B161
:1075F00084F83CA001E084F83C60204608F00EF8D6
:1076000048B185F814800421204601F03FFE38B9C6
:1076100084F831A002E0042184F83110C4F8A49069
:10762000A07878B13A4604F15400D4F8A41072DF7F
:1076300000287FF405AF94F8301094F8540073DFFD
:107640000028F6D1616B11B194F831008847002011
:10765000F6E684F83150F5E770B5040012D0014623
:107660001C221448FEF702FF1248134D05602068E3
:1076700050B17ADF002806D120680168296040688F
:10768000686005E00E2070BD0B487BDF0028FAD152
:1076900008484FF6FF711438084A20F8041B0549C2
:1076A000343901600021FFF73FFB0028EBD00320B5
:1076B00070BD0000AC25002040220020B5F502007E
:1076C00010B5044600F078F8002805D02146BDE842
:1076D0001040024803F017B910BD0000D825002063
:1076E00070B515460E46044607F0A4FF002809D0E1
:1076F000054800EB840080692A463146BDE87040A9
:1077000001F002BE70BD0000C825002070B505461E
:10771000002400F051F838B12946044803F0F3F88A
:1077200008B1022400E00124204670BDD4250020C9
:1077300010B51821034803F0C1F8182800D0C0B2D2
:1077400010BD0000C825002070B505460C4608464F
:1077500007F070FF60B1284600F02EF840B10548F0
:10776000294600EB8400BDE87040183003F0CBB828
:10777000002070BDC825002070B5054614460E4691
:10778000084607F057FF002812D0284600F014F8EA
:1077900000280DD00748294600EB860018301CB1A0
:1077A000BDE8704003F0BAB8BDE8704003F06BB8B4
:1077B00070BD0000C8250020142801D300207047A8
:1077C0000146014803F09FB8CC2500207CB5054652
:1077D00008880C460930904201D90C207CBD6846CF
:1077E0006DDF0028FAD121880820685420881B21E9
:1077F000401C80B2208029542088401C80B2208008
:107800002844DDF801100160BDF805108180208852
:10781000801D80B220809DF80010490800D0012111
:1078200029542088401C208000207CBD10B503F026
:1078300055FA002809D105484FF0020C00DF002856
:1078400003D1BDE8104003F0ADBA10BDB828002048
:1078500020B103490860034806F0EABA0E207047D9
:10786000A022002001DA020010B54FF0FF31002005
:107870003DDF00280BD1B1213CDF002807D10448AF
:10788000416901208847022004F0AAFB002010BDB6
:107890009C28002070B50E4C206841690020884764
:1078A00020681321808876DF050008D0094801216F
:1078B000008801EB004008A104F0B8F905E005F0EC
:1078C00031FF2168086101F083FF284670BD000088
:1078D000A0220020242400204661696C6564207485
:1078E0006F20646973636F6E6E65637420474150E7
:1078F00020636F6E6E656374696F6E0030B58FB014
:1079000005461C2101A8FEF7CAFD0024142109A880
:107910000894FEF7C4FD9DF82000009420F00F00AD
:10792000401C20F0F00010308DF820009DF8210060
:10793000029420F00F00401C20F0F00020308DF861
:1079400021009DF82200049420F00600801C8DF890
:1079500022009DF8040009AA40F028008DF80400D8
:1079600008A8CDE90540079428788DF83A0004204E
:10797000ADF838009DF80000ADF82C4020F00F0065
:10798000401C20F0F00010308DF800009DF8010040
:10799000ADF82E4020F00F00401C20F0F000203009
:1079A0008DF801009DF802000D9420F00600801C67
:1079B00020F0080040F011008DF802000EA8099098
:1079C0001720CDF828D0ADF830006888AB1D01A98C
:1079D000AADF0FB030BD000010B5164C86B01ECC2B
:1079E0008DE81E0020B3144C4FF6FF71A180006893
:1079F00060610020607620762046FFF729FF00288E
:107A000014D101208DF812004FF65960ADF8100026
:107A1000A21C04A90120A8DF002807D1214668463E
:107A200062DF002802D12046FFF768FF06B010BDD4
:107A30000E20FBE7F0FC02009C28002010B5002877
:107A40000FD00188204C502926D00BDC10291DD0E6
:107A5000112906D1A1888088814202D14FF6FF709A
:107A6000A08010BD512913D05329FAD1C088E188D4
:107A70008842F6D1607E0028F3D0FFF70BFF002884
:107A8000EFD06169BDE81040022008478088E7E731
:107A9000BDE8104005F07AB930F8061F62899142BE
:107AA000DFD141890229DCD10C3000F0BDFA074951
:107AB000207603220988BDE8104002EB014302460C
:107AC00003A1184604F0B6B89C2800202424002006
:107AD000526563656976656420696E646963617483
:107AE000696F6E2073746174652025640000000066
:107AF00070B50546007B0424012810D00224287BA1
:107B0000214600F051F80C4C18B12068416903205F
:107B1000884720684169BDE870400220084701F0AD
:107B20006BF8002807D0112803D00F28E7D10724CD
:107B3000E5E70624E3E770BDA022002070B51849F0
:107B400000250A68002A2AD04A68002A27D0012680
:107B500008319047082822D0124C0028206810D005
:107B6000457685760621012000F01EF818B12068C0
:107B700041690320884720684169BDE870400220C0
:107B80000847467685760121084600F00DF8002862
:107B900005D020684169032088472068457670BD7C
:107BA000B8280020A022002086B00323ADF80030C2
:107BB00020238DF814308DF8150000220E48019214
:107BC00002928DF81610C188ADF8041002218DF8CC
:107BD000061005A90491ADF80820CDF80CD08088D6
:107BE00001A9AEDF002804D1BDF80010032900D0A0
:107BF0000C2006B0704700009C2800200F4A03218B
:107C0000128801EB024268B101280ED00B4A012113
:107C10000228128801EB02420AD0032810460AD03B
:107C200007A109E0104610A106E010461AA103E0E2
:107C3000104622A100E030A103F0F8BF2424002068
:107C4000556E6B6E6F776E206576656E742066720A
:107C50006F6D20626C655F6466755F627574746FCA
:107C60006E6C6573732E00004465766963652069E8
:107C70007320707265706172696E6720746F206521
:107C80006E74657220626F6F746C6F6164657220D0
:107C90006D6F64652E00000044657669636520772A
:107CA000696C6C20656E74657220626F6F746C6FA6
:107CB00061646572206D6F64652E00005265717598
:107CC00065737420746F20656E74657220626F6FC7
:107CD000746C6F61646572206D6F646520666169A4
:107CE0006C6564206173796E6368726F6E656F7521
:107CF000736C792E000000005265717565737420F5
:107D0000746F2073656E64206120726573706F6E8E
:107D1000736520746F20636C69656E742066616999
:107D20006C65642E0000000038B5044600882128E8
:107D30001CD013DC102822D1072000F0E1FA08B192
:107D4000FEF7A0FF1048A1880180104802F03EFF16
:107D5000002814D0BDE83840FEF794BF3B280FD070
:107D600056280CD1A088132176DFF1E7002000907F
:107D7000A08869468FDF002801D0FEF783FF38BD59
:107D8000A088132176DFE3E720220020482400208A
:107D900010B51A4C0188606810290ED011292BD11A
:107DA000401E606028D1FEF770FE002824D02168B4
:107DB000002921D0BDE810400847D0B90021012298
:107DC000084600F07BFA08B107280FD107220221EC
:107DD000012000F073FA08B1072807D1042202211C
:107DE000002000F06BFA20B1072802D0216801B111
:107DF00088476068401C606010BD00003822002089
:107E00002DE9F04701883B4E40F2F3194FF6FF751C
:107E100010291BD011293ED0122954D0502946D107
:107E2000C188F289841D914241D1618902293ED1E4
:107E30008688304601F0B2FF050038D004F10C000E
:107E400000F0F6F8A8B3294630464EE0C17B87889B
:107E5000044601292BD1A846284601F09FFF0500C2
:107E600017D02F8000202872234843464A460168D5
:107E7000C5F80A104068C5F80E0004F1100105F1BC
:107E80000A0002F057F86872F08900280FD12946DD
:107E90002AE0042013E0808801F080FF040006D06F
:107EA0006068FEF7C1FF08B106F094FC2580BDE8CC
:107EB000F087FFE76868FEF7B7FF0028F7D0BDE856
:107EC000F04706F087BC87880646384601F066FF13
:107ED0000400ECD02B464A4606F1080104F10A00E2
:107EE00002F028F8607221463846BDE8F04700F0FD
:107EF000E3BC0000AC250020402200202DE9F04F1B
:107F00000746858802883D48012197B08346102A9C
:107F100009D0112A49D01A2A6CD1387AB1EB101F36
:107F200045D2012244E0354C083CA068C0430B9088
:107F300061680BA802F00BFD0B990CA800F056FC31
:107F40002C220CA96846FEF791FA0026E946A046C5
:107F500010E000BF09EB46005FF00004B0F804A099
:107F600008EB84005146001D02F08DFC641C1D2CA2
:107F7000F6D3761C0098B042ECD8142D05D317B078
:107F80000420BDE8F04FFEF77DBE2946584602F0BA
:107F9000C5FC294608F1040002F0C0FCF87B01286A
:107FA00028D016482946001D15E029461AE000226F
:107FB0000221B1EB101F01D2012600E000260F497B
:107FC000083901F11000041D294682B102F0A6FC17
:107FD00036B12946204617B0BDE8F04F02F09EBCEE
:107FE0002946204617B0BDE8F04F02F04CBC02F025
:107FF0004AFCF5E717B0BDE8F08F0000D02500205F
:1080000010B504460748007800280AD0204601F041
:10801000F3FC204606F038FD2046BDE8104001F094
:108020007FBA10BD702200200078C0F34000704776
:10803000007800F0010070470149085C70470000BB
:10804000A8FB0200084908B5085C0090684603F0E8
:1080500073FBD0F810050099C84010F0010000D063
:10806000012080F0010008BDA8FB02002DE9FC41C1
:108070000646C0074FF000050ED0104F0024012225
:10808000385D009500231146019503F0A1FA641CA8
:10809000042CF4D300F04EF8B0070DD5074E0024A1
:1080A000361D0022305D032300951146019503F033
:1080B0008FFA641C042CF4D3BDE8FC81A4FB0200FD
:1080C000094908B5085C0090684603F035FBD0F814
:1080D0000425009B0121994021EA0203C0F80835DC
:1080E0001140C0F80C1508BDA4FB02000249085C51
:1080F000012103F078BB0000A4FB02000249085CE8
:10810000002103F070BB0000A4FB0200084908B581
:10811000085C0090684603F00FFBD0F80405009956
:10812000C84010F0010000D0012080F0010008BD1F
:10813000A4FB020010B500242046FFF7D7FF641C03
:10814000042CF9D310BD10B500242046FFF7D6FF4C
:10815000641C042CF9D310BD10B50246064B4FF039
:10816000FF3000215C5C944201D1084610BD491CDF
:108170000429F7D310BD0000A8FB020070B50C4E17
:108180000C004FF0000530600BD0012000F06AF8C1
:1081900008B1022004E0002000F064F800B10B20D8
:1081A0002070706810B9FEF770FC0546284670BD57
:1081B0003822002010B5002000F0D4F908B10628BC
:1081C00006D1012000F0CEF908B1062800D1002028
:1081D00010BD00002DE9F0470D468146FFF7BCFFBA
:1081E0000446042836D2DFF874801B481C4EA8F1E0
:1081F0000C0725B3012D0ED0022D2BD104EB44002A
:1082000030444578002D25D0B968002922D0284671
:10821000BDE8F047084704EB4401755C0E447178F3
:1082200049B10E4A4FF40041093A8068FEF7B8FDA3
:1082300008B987F80390B17808F80410E2E780687D
:10824000FEF7F2FD04EB4401314418F804008D7888
:10825000A842D7D0BDE8F087ACFB02003422002052
:108260004C250020042801D2FFF7ECBE0020704707
:108270000146104810B50088042907D007290ED000
:108280000A2915D1BDE8104006F0E8BB132176DFBE
:108290000CE000280CD0BDE81040FEF7F3BCA0F5C0
:1082A0007F41FF3904D10448FFF79EF80828F0D138
:1082B00010BD0000202200205424002070B50023AF
:1082C000042810D20D4D00EB4004012A02D10129EF
:1082D0000CD00022094E00EB4000304461B101296E
:1082E00006D0022906D00723184670BD0E30C2B250
:1082F0002A55F9E74270F7E78270F5E74C25002030
:10830000044A014600201279D20702D0084600F044
:108310004DB870472822002070B506461E4800243C
:10832000C0E90161B00720D5002501221146284689
:10833000FFF7C4FF6D1C0446042D02D2002CF4D0BC
:1083400013E094B940F2666204211448FEF720FC61
:1083500004000AD1FEF70AFC040006D10F48104AB7
:108360000021001FFEF7E0FC0446F00712D00120B8
:10837000FFF77CFE74B909480A4A00210C38FEF761
:10838000D3FC040006D10548074A01210838FEF74E
:10839000CBFC0446204670BD28220020B8FB02001A
:1083A00031860200C99F02005B6B02002DE9F05F7D
:1083B0006A4C054600266078B34618B184F801B0CF
:1083C00001F0EAFD664F4FF47A694FF4C87A4FF036
:1083D0000108182D62D2DFE805F0AC0C0C31404DDD
:1083E00062676B746B74BE7D7D7D7D7DACAFB2B515
:1083F000BEBE0020FFF78AFE00284FF0000008D024
:10840000FFF774FE022D02D14FF4E16008E0484608
:1084100006E0FFF773FE022D01D1C82000E05046B0
:10842000410CC0034FF4FA72801841F1000125702D
:1084300052000023FDF7D6FF01462AE00020FFF797
:1084400065FE00284FF0000004D0FFF74FFE4FF408
:108450004870E5E7FFF752FEDFE70020FFF756FE22
:1084600000284FF0000002D0FFF740FECFE7FFF7F3
:1084700045FED4E70020FFF749FE00284FF000003A
:1084800002D0FFF733FE01E0FFF738FE257041F61A
:108490009A1100223868FEF783FC064646E0002069
:1084A000FFF70EFE257008E0002051E025703DE04A
:1084B00084F801800120FFF703FE002240F6CD4141
:1084C000E8E784F801800120FFF7FAFD00224FF46D
:1084D0008041DFE77868FEF7A7FC0646D5F111007A
:1084E00000D02EB10220FFF701FE84F802B01DE09B
:1084F000012816D980B2C8214843C117C90341EAEF
:108500005041C0034FF4FA72801841F1000152004B
:108510000023FDF767FF014600227868FEF740FC64
:1085200006460220FFF7EAFD84F802803046BDE8E7
:10853000F09F01F031FDB9E701F02EFDB4E701F045
:108540002BFD04E001F028FD0020FFF7D7FD0120FE
:10855000FFF7D4FDAAE7FFF7F6FDA7E728220020E2
:10856000ACFB0200012107F0FDB800002DE9F84343
:108570000546861C00208DF8000090460F464FF0FF
:1085800001096846FEF760FC1B4C20683860D4E99E
:108590000001401AA16804F21C47081A0EE00121EC
:1085A000384602F0CEF901F0ADFE0146384602F041
:1085B000C8F9D4E90001401AA168081A401C864293
:1085C000EDD8B8F1000F03D0052065F3891002E063
:1085D000062065F39F50A2682168114004EB8101D9
:1085E000C8602068304420609DF80000FEF750FC11
:1085F0004846BDE8F8830000B82D002030B48268FA
:108600000468531C8360A154D0E901128A4202D34A
:1086100030BC02F08ABC30BC70470000034803C87D
:10862000814201D10120704700207047B82D002001
:1086300000780221FFF7CEBD032805D10349A92008
:108640000860002003F0CCBC70470000200500400B
:1086500005494FF0FF32082841F8202002D3084492
:1086600080F858207047000018290020F0B54FF01E
:10867000FF3512B10023082601E008230C260C4C1C
:1086800005E000BF54F823707F1C04D05B1CB3428C
:10869000F8D32846F0BD26185DB286F8305044F86D
:1086A0002310002AF5D1E11881F85800F1E7000005
:1086B000182900200249084490F930007047000052
:1086C0001829002070B504464FF6FF750A46284663
:1086D000AC4208D14FF480742146104605F0F0F901
:1086E000A04209D070BDFF2CFCD82146104605F0F1
:1086F000DAF908B1204670BD284670BD70B5084C47
:10870000050009D010342168002907D008682060CE
:10871000496828468847F6E70834F4E770BD00004A
:1087200004290020054A012120B1012805D19170BA
:10873000FFF7E4BF51700020FAE7704704290020DA
:108740002DE9F05F26484168F1B3DFF898B00E6874
:108750008146DBF8004087688078E11B21F07F4587
:10876000ED1CB0B9DFF880804FF48030C8F84403C6
:10877000C8F804031120FDF7D9FF1120FDF7E1FF30
:108780004FF0010AC8F800A02F2003F0EBFE89F893
:1087900002A0B54200D23546124BE8193C3320F016
:1087A0007F401860DBF800105A46091B21F07F411A
:1087B000001B20F07F40C91C81420FD9106818604F
:1087C0002F2003F0CFFE00E004E0BDE8F05F1120B1
:1087D000FDF7C2BFBDE8F05F05F020BEBDE8F09F29
:1087E000E8220020041501400010014073B58CB050
:1087F0000646002000900D9880B100246D46214669
:108800000DA802F080F830B1009805EB400084809C
:108810000098401C0090641C142CF0D32C22694654
:108820003046FDF723FE0EB070BD2DE9F0411788EC
:108830000646B81D14460D46984202D90C20BDE8E4
:10884000F0813188072206290AD34FF4486C4FF68D
:10885000FF73614501D9994202D17088062801D27F
:108860001046ECE7604501D99842F9D1994203D00E
:10887000984201D08142F3D80520E8552088122182
:10888000401C80B2208029542088401C80B2208067
:108890004119308806F014FE2188084480B22080F7
:1088A0004119708806F00CFE2188084420800020C1
:1088B000C5E7FEF7E7B9000038B54A7A0F4B62B159
:1088C00000220A725969002906D001228DF8002081
:1088D000ADF802006846884738BD0A7A62B19B68E5
:1088E0004C68024619462046FEF75AFA0028F3D093
:1088F000BDE8384005F06EBF5B68F1E7AC250020AD
:10890000F0B585B016460F4604461D4614220B49A5
:108910006846FDF7ABFD0A488DF80870ADF80240D7
:10892000ADF80A608DF80C50017800222046FEF761
:1089300023FF684600F0A4FA05B0F0BDC4FC0200B5
:1089400080220020F0B587B0074600200490ADF8E3
:1089500010100590ADF812100190029001AA04A920
:10896000384690DF060022D003F0A2FD114C0346EA
:10897000012520883A4605EB00400F4903F061F9D4
:10898000BDF8042012B9BDF8060038B12088BDF842
:10899000063005EB004009A103F053F9BDF80820AB
:1089A0002AB12088154905EB004003F043F907B0D0
:1089B0003046F0BDF42300209C000300546865207D
:1089C0007265717565737465642054582F52582010
:1089D0007061636B6574206C656E67746820697381
:1089E00020746F6F206C6F6E672062792025752F61
:1089F0002575206F63746574732E0000E800030012
:108A000030B5044685B000211B4805F04CF800281D
:108A10002FD00025204600F01EFF68B1112812D08B
:108A200086281BD0A0F54051023903D001462046CC
:108A300005F0D8FE294607E005B029462046BDE8E6
:108A4000304001F03DBC0121204601F039FC05B069
:108A50000021BDE83040084805F059B81422074904
:108A60006846FDF703FDADF80240684600F0E4F902
:108A7000E0E705B030BD000049220020ECFB020019
:108A80007FB50C4610B1012004B070BD20790026DE
:108A900038B141F61D5501281BD0022826D00F20E1
:108AA000F2E70220207102960396E0680190694681
:108AB00001A805F0D7FB50B102988188E1800088B9
:108AC0002081BDF80010029805F04AFCDCE70A207E
:108AD000DAE70A4B6A460021A01D05F07FFB38B19A
:108AE000064918398E61CE610A28CDD12846CBE7D8
:108AF00002488188019805F033FCF5E7282300201F
:108B00002DE9F0470025DFF88C803CE0606800210B
:108B100000EBC506012032789146FDF794FCD4E9BC
:108B2000062300EA020701EA030C57EA0C0728D0E3
:108B300082438B434846C4E9062303F0D1FD3278D3
:108B40008246914601200021FDF77DFCD4E90423F3
:108B500000EA020401EA03074A4650460021FDF7F5
:108B600072FC44404F403C430BD17078012801D047
:108B7000012100E00021726881EA0A010AB1484639
:108B800090476D1CEDB298F8000044468542BDD375
:108B9000BDE8F087C822002010B50021024801F08E
:108BA000EBFE80F3100010BDD43100200E4910B54B
:108BB0000A784C780023A24212D0521CD2B20A701A
:108BC000022A00D10B70084A0B780C3252F823208D
:108BD00002608868104420F07F408860012010BD4A
:108BE0000360002010BD0000E822002013460A4662
:108BF0000021FFF785BE000070B5174D03212888BE
:108C000001EB004015A103F011F81E4E3068807E84
:108C100028B1BDE8704006210120FEF7C5BF05F070
:108C2000C3FB002816D11848A0F10C010A68011FE7
:108C3000904704004FF0010002D00F2C03D008E051
:108C40003168887605E0298800EB01400F4902F081
:108C5000EDFF204670BD0000242400205772697487
:108C6000696E672070656572206461746120746F3D
:108C70002074686520626F6F746C6F616465722E1A
:108C80002E2E0000A0220020C42800204001030056
:108C90002DE9F843104D0F4680461E469146694621
:108CA000286801F0C4FD040014D01C21FDF7F7FB77
:108CB00001202071C4F81490380BC4F80080C4E976
:108CC00002606946286801F0D3FD05F01BFA002018
:108CD000BDE8F8830420FBE7B0FD020010B503787F
:108CE0000022072B06D2DFE803F005040610202936
:108CF00030000A7010BD01230B7003898B818388BB
:108D0000CB81C06888600A7410BD02220A70028993
:108D10008A818288CA81C2688A60807D062802D0E2
:108D20000020087410BD0120FBE703220A70C288EE
:108D30008A810289CA81C068886010BD04230B70D3
:108D4000C0888881CA818A6010BD0520087010BD66
:108D500070B5064D0646002455F8241009B130467A
:108D60008847641C042CF7D370BD0000182B00202A
:108D700030B50446006887B00D46806800281FD0D3
:108D800018216846FDF78BFB0195A06805902079B6
:108D900010B1012810D107E001208DF800002069F2
:108DA0000290E068039005E002208DF80000E06882
:108DB00000030290606904902068816868468847D3
:108DC00007B030BD70B586B015460C00064619D008
:108DD000112C17D0082C15D014216846FDF75FFB25
:108DE000ADF80260304600F02DFFADF804000D2C08
:108DF0000AD0862C1CD007208DF80000029468460B
:108E000000F04CF806B070BD03208DF8000025B1CD
:108E10002878C00701D0012000E002208DF808006A
:108E200000208DF80C0041F20110ADF80A00E6E7D1
:108E300006208DF80000E2E710B50446408800F0F7
:108E400001FFA080024801682046BDE810400847A5
:108E5000502200202DE9F04107460024064E074D20
:108E600005E000BF56F8241038468847641CE878AF
:108E70008442F7DBBDE8F0815028002070220020FA
:108E800010B50446408800F0DDFEA080024801686D
:108E90002046BDE81040084798FC020001490968D7
:108EA00008470000ECFC020070B586B004461421AF
:108EB0006846FDF7F4FAA0890125A0F54040ADF819
:108EC000040020782A4E062833D2DFE800F032036F
:108ED00003032C48A08900F0BDF930B9E08943F6BE
:108EE000FE71A0F54040884223D8A07B8DF8080091
:108EF000207803280FD000208DF80900A068039087
:108F0000606850B109208DF80000606804906846E0
:108F100004F0FAF90DE00120EEE708208DF80000DA
:108F20008DF81050F3E7A08900F094F908B1E089BA
:108F300030B17078002801D004F016FB06B070BD87
:108F4000606820B10B208DF800007570DFE70A2003
:108F50008DF80000BDF8040004F090FBF5E7132045
:108F60008DF800004FF6FF70ADF80400CFE7000069
:108F70006022002038B504460E480078A8B1A4F558
:108F80007F40FF380FD0684604F0EEFF78B105212E
:108F9000017001210171C480684604F0F3FF05F0FF
:108FA000A3F8002038BD042038BD022038BD0820B9
:108FB00038BD0000302300200C4808B5007888B187
:108FC000684604F0D1FF78B106210170684604F0CC
:108FD000D9FF0748017809B10121017305F084F830
:108FE000002008BD022008BD082008BD3023002055
:108FF000DC2B0020F0B587B014216846FDF74FFA4E
:109000002B4C207818B16846FFF7A2FE4EE0201DD9
:1090100001F094FCB8BB4FF01020416900040269D4
:1090200040694B1C01D100FB02F122480022016182
:10903000A1F54051C160204902F006F9002820D175
:109040001F481C238C221D49006801F0DDFB03F042
:109050004BFF051E14D0022812D000270126062D32
:1090600012D005A804F080FF88B106700C2D18D22C
:10907000DFE805F0170F170F171617161711131142
:109080000B2007B0F0BD11E026706760BBE7082039
:10909000F7E7077105E0032100E00221017100E01C
:1090A000067105A804F06EFF05F01EF80020E8E741
:1090B00030230020E0230020C0FD0200282B0020E8
:1090C00028FD020038B5040014D0694605F0CAF83E
:1090D000A0B1BDF8000000EB8001094800EB810061
:1090E000C16849B1A17A39B1C168491EC160002087
:1090F000A07238BD052038BD062038BD0A2038BD15
:10910000B42B00201FB501A9684605F067F804B02C
:1091100010BD07B513460A466946002005F05EF803
:109120000EBD07B513460A460021684605F056F8FD
:109130000EBD20B119B100680860002070470520FD
:1091400070470000F8B50D46040018D0BDB169465F
:1091500005F088F8A8B1BDF800000B4900EB8000CD
:1091600001EB800001210C30666801F0EAFB2E6003
:1091700060680C3068600120A0720020F8BD0520F6
:10918000F8BD0A20F8BD0000B42B002018B103235D
:10919000002206F0DFBB052070470223002206F004
:1091A000D9BB12B1022306F0D5BB052070470000E1
:1091B000084910B50A69042A0AD0074A096942F821
:1091C000210004480121103001F0BBFB002010BD3C
:1091D0000C2010BD10230020182B002038B50446A9
:1091E00009480D46007858B164B16946284606F032
:1091F000ABFC002803D1BDF800102180658038BD8C
:10920000022038BD052038BD3023002010B50446AB
:109210000E48007898B1A4B12188022913D80C4ACD
:1092200001EB810002EB800260885289C31C9342EB
:1092300009D806F07DFC00202080608010BD02204F
:1092400010BD052010BD042010BD000030230020FB
:10925000B42B002043F6FE71A0F54040884201D8AF
:10926000012070470020704710B504460078182888
:1092700002D1FEF75DFA207010BD10B504460078EB
:10928000182802D1FEF754FA207010BD70B50D46B3
:109290000446B0F89810D0F894000122FDF7B3FF0F
:1092A00000B1057004F13C0204F1940104F1540092
:1092B00072DF70BD70B5134600220646154686293A
:1092C00002D0112902D002E0012200E001250D4C5C
:1092D00073B1A179FEF750FA2A4661793046FEF75C
:1092E0004BFA0022A1783046FEF746FA002203E04E
:1092F000A178FEF741FA2A4661783046BDE8704011
:10930000FEF73ABA88220020F7B517460E0011D0B2
:109310000098002560B100242146684601F0F3FA68
:1093200018B1A0B23946B0476D1C641C142CF3D39D
:109330002846FEBD0020FEBD406804F035BE00009A
:1093400070B508B1012070BD194C0025207B08B113
:10935000257301E000F0A0F82078082826D2DFE885
:1093600000F02504080C10251420BDE8704000F022
:1093700021B8BDE8704000F07DB8BDE8704000F055
:109380005FB8BDE8704000F03BB86088084900EB6A
:109390008000283901EB80004068BDE8704003F090
:1093A00083BD6560BDE8704003F08CBD0F2070BDCB
:1093B000DC2B00201149F0B48A1C00200346A1F1E7
:1093C00028050C18A67A4EB1A37200EB800405EBB9
:1093D0008404E66816B9247C012C0AD0401C80B2B3
:1093E0000228EED30B704B804B60F0BC41F61D5051
:1093F00070471080F0BC00F03DB80000DC2B00206E
:109400000C48418801EB8102A0F1280101EB8201A7
:10941000CA6852B1052101700748022181800168A4
:1094200000230122054801F079BE04220270496838
:10943000F6E70000DC2B002038230020E02300208A
:1094400038B50A49084803240B684268898803EB49
:10945000810153880470DB1C00201B0400909B0BCF
:10946000034801F0CBFF38BDDC2B0020382300205F
:10947000E0230020074910B54888091D04F042FF89
:1094800018B1BDE81040FFF7DBBFBDE81040FFF7A3
:10949000B7BF0000DC2B0020F0B51F481F49012595
:1094A000067802248B88A0F12802082E19D2DFE862
:1094B00006F00418181B222F2F170189491C01815F
:1094C0000021418080F80C1001EB810312F8233059
:1094D00043B100234418491C89B2A3720229F3D373
:1094E0000570F0BD0123F5E742685288D21C1A448A
:1094F0008A800470F0BD46880D6806EB860602EB94
:10950000860256680E60556013818C80062100E04B
:1095100007210170F0BD0000DC2B00203823002063
:1095200030B501888488224D85B0502924D0522935
:1095300002D0542931D103E0204600F08DFE2CE00A
:1095400014221C496846FCF791FFADF80240204602
:1095500000F078FBADF8040000F022F900226979F0
:109560002046FEF709F9002229792046FEF704F982
:109570006846FFF761FC10E0017B01290DD1817A7B
:1095800001290AD10089A0F52451023905D1012110
:10959000204600F095FE06F003F800220649E87820
:1095A000FEF79EF805B0BDE8304005F063B9000055
:1095B0004822002014FC0200B16F020010B50446DE
:1095C000007800280FD1608800F046FE608800F027
:1095D0008FF9002807D00449608801220979BDE885
:1095E0001040FEF7C9B810BD4822002010B5124C3B
:1095F00000202070FEF79CF8A070FEF799F8E0704C
:10960000FEF796F82071FEF793F86071A17818299B
:109610000FD0E17818290CD02179182909D0182801
:1096200007D00121601C04F037FA012020700020CF
:1096300010BD032010BD0000482200207CB5044668
:10964000007808282FD1607A38BB207A4FF6FF7552
:1096500001280DD0072802D0082824D11EE0A088B8
:1096600000F02EFAA8421ED0012100F029FE1AE0D7
:10967000A0886A46012103F05FFD70B90198007867
:1096800058B1A08800F01CFAA8420CD00849012269
:109690000979FEF771F805F0EDF804E004480021BF
:1096A000401C04F034FABDE87C4005F079BF0000AE
:1096B0004822002010B504460A4841782046FEF7AB
:1096C00043F868B10848002101EB410200EB820237
:1096D0005288A24201D1C8B210BD491C1429F3D34B
:1096E000FF2010BD5A2200204026002070B5094DF1
:1096F000094E002404EB440005EB8000717840889B
:10970000FEF722F820B1641C142CF3D3FF2070BDA7
:10971000E0B270BD402600205A2200202DE9F04121
:109720008046024601200021FCF78DFE1A4F0546B7
:109730000E467868FDF778FB00280CD1174CD4E969
:10974000062110462A4001EA06031A4305D0A84321
:10975000B143C4E90601BDE8F081404602F0C0FF14
:1097600030B1D4E9040128433143C4E9040105E0E0
:10977000D4E90410A943B043C4E90410D4E90601B4
:1097800028433143C4E90601A1687868BDE8F04187
:109790000022FDF705BB000010FD0200C8220020DA
:1097A0001CB5054AD2E90212CDE900120022694631
:1097B00003F0E7FC1CBD00002CFC020003484FF640
:1097C000FF71818001210170002070475422002028
:1097D00010B54FF6FF7003F069FC03498880BDE8BF
:1097E000104005F051B80000542200202DE9FC4142
:1097F000804600F027FA002403250127A0F57F41C9
:109800002646FF3908D06A46082103F095FC18B9AE
:109810000198841D8688056832462B4621464046BD
:10982000B1DF042804D0082804D00B2808D002E0B7
:10983000112000E00020002F00D10B20BDE8FC81AA
:109840000027A80701D50125E6E73443F5D0002419
:1098500026460325E0E72DE9FC41804600F0F2F9B9
:109860000646A0F57F40FF380ED001252A466D1C24
:109870000027ADB26B460821304603F087FC040098
:1098800006D0072C25D025E043F20200BDE8FC817C
:10989000019903230A1D0B604046891DB2DF0400B5
:1098A00004D00C2C09D0052C09D009E0324608213F
:1098B000104603F0E1FC04460CE0012700E0002420
:1098C0000821304603F0C4FC00B10324002FCDD1A1
:1098D00000E00C242046D9E704488088A0F57F41A9
:1098E000FF3901D004F0D0BF70470000542200209F
:1098F0000EB502A9019100F0A5F96A46012103F015
:109900001BFC08B100200EBD019800780EBD0000C0
:109910002DE9F04107464FF6FF760A48B3DF10B154
:109920000320BDE8F081074C43F20305A41E324634
:1099300061883846AFDFA842F3D16088401C608060
:10994000F5E7000056220020428800EB82020C322C
:109950008A4201D9022070478188A1F57F42FF3AEF
:1099600003D0008808B1002070470120704788426A
:1099700004D20068401C01D00120704700207047CD
:109980003EB5027802230C46B3EB520F17D1B0F864
:109990000110ADF80010C1788DF802108188ADF883
:1099A000041080798DF8060002AA01A92046FDF76F
:1099B000ABF8032202A96846FCF783FD08B100203A
:1099C0003EBD01203EBD000010B50C46FFF772FE03
:1099D000FF280CD0074900EB400001EB80004168F4
:1099E00021600189A180807AA071002010BD05202E
:1099F00010BD00004026002070B5018890B01029ED
:109A000059D1011D2C226846FCF730FD9DF8040059
:109A10004FF6FF76032134466D46B1EB500F2AD046
:109A200003F0E0FC9DF8040040080ED001280CD0A3
:109A3000022820D118E00D99281D1131FDF700F8FA
:109A400018B100BFBDF82C4015E00CAA0BA90720E7
:109A500003F09CFC0028EED10DE00D99281D491C57
:109A6000FFF78EFF0028EDD10CAA0BA9072003F009
:109A70008DFC0028F1D1BDF80000291D00F06EFE1C
:109A8000B44218D0BDF80000214600F0C5F8BDF87A
:109A90000000ADF82E000020ADF83040074E8DF8E4
:109AA0002C000BAD044600BF56F82410284688470A
:109AB000641C022CF8D310B070BD000040FC020002
:109AC000094A002101EB410332F82330834205D1DA
:109AD00001EB410002EB800040887047491C1429CB
:109AE000F0D34FF6FF707047402600203EB50C467D
:109AF000054603F077FC0BE0BDF80000A04207D05C
:109B00002846029900F02EF810B1BDF800003EBDC5
:109B100001AA6946072003F039FC0028ECD14FF672
:109B2000FF703EBD10B50D4C18200D4A607000202E
:109B30004FF6FF7100EB400302EB8303401C59809A
:109B40001428F7D3FDF7F4FD6070182803D0012026
:109B50002070002010BD032010BD00005A220020FC
:109B6000402600202DE9F0410C46054600F1110782
:109B700001F111061022491C401CFCF7A2FC48B957
:109B8000681C00F0F9F928B1601C00F0F5F908B183
:109B9000012400E0002431463846FCF751FF3B78B1
:109BA0000222B2EB530F0CD00321B1EB530F08D0BC
:109BB0003378B2EB530F04D0B1EB530F01D0012136
:109BC00000E00021084201D18C4302D00120BDE811
:109BD000F0810020FBE7018811B9421892780AB1A0
:109BE00001207047491C0829F7D30020704710B5A1
:109BF0000C460346FFF7EFFF00280AD0188821889B
:109C0000884205D10822A11C981CFCF75AFC08B117
:109C1000002010BD012010BD03F094BD70B50446B6
:109C2000FFF74EFF0546204603F089FA4FF6FF7115
:109C300004468D4203D014B9284603F083FD204624
:109C400070BD000010B5FFF735FDFF2805D00449B1
:109C500000EB400031F8200010BD4FF6FF7010BD42
:109C6000402600203EB5044603F0BCFB0EE00199FF
:109C700020464631FFF7BBFF28B9019920462A311B
:109C8000FFF7B5FF10B1BDF808003EBD6A4602A956
:109C9000072003F07BFB0028E9D14FF6FF703EBDA3
:109CA00010B50A4941600A4800F048FE58B902F070
:109CB00089FB07491C238C22087404488C39001F37
:109CC000006800F0A1FD002010BD0000B4FD0200FE
:109CD000782C00202DE9F0412D4F002518B17D6032
:109CE0000120BDE8F0810879012258B1294E0128F0
:109CF0000CD0274C4FF002080834022821D003284A
:109D000042D128E00A7103F0DDF83BE05FF000008B
:109D100000EB800116F82110022908D0401C80B207
:109D20000228F5D33A707D6041F61D50D9E700EB6B
:109D3000800006F8205006EB8000406803F0B4F87D
:109D400020E00D71A4F8048000230122124821684C
:109D500001F0E4F916E00D71206803F0A5F80D4953
:109D600023682831498801EB810206EB8201D1F892
:109D700004C0C4F800C04B60A3880B81A4F8048021
:109D800006F822500028ACD07D600E20A9E7000024
:109D900030230020B42B0020E0230020014603489C
:109DA00002888A4200D000207047000098250020D9
:109DB0002DE9FC5F0E008346DDE90C47C6F100008B
:109DC00098469246814600D40846012503E000BF2C
:109DD00090FBFAF06D1C5045FADAA84500D94546CB
:109DE00024B1002E01DB780700D5641EB80702D528
:109DF000B8F1000F0AD0F80708D13CB1A54205D24E
:109E000020215846641EFEF7F9FBF6E7002E02DA21
:109E10004E462D2102E0780703D52B215846FEF748
:109E2000EDFB07F0030002280BD1B8F1000F08D1B9
:109E30003CB1A54205D230215846641EFEF7DEFB38
:109E4000F6E7CDE90047434652463146584605F00D
:109E50004DFBBDE8FC9F000070B50D460446006850
:109E60004FF4887102F044FB4FF49071206802F0C7
:109E70003FFB4FF49271206802F03AFB4FF4A2715D
:109E8000206802F035FB20681249C0F804132068EE
:109E90006907000B40B2090E002806DA00F00F0037
:109EA00000F1E02080F8141D03E000F1E02080F8CC
:109EB000001420680121000B40B200F01F02914005
:109EC0004009800000F1E020C0F88012C0F80011C5
:109ED00070BD0000100302000246002012689307C4
:109EE00002D0530702D47047500714D502F0030084
:109EF000012802D002280CD105E0C2F383100B68C0
:109F0000801C184404E00223086803EB92521044BA
:109F1000086001207047086800EB9253C2F3891073
:109F2000401CEEE70248007A002800D0012070476C
:109F3000782C0020F0B58488A518944200D82246D9
:109F4000A41AC288D6189A4200D81346D21A4B884F
:109F50000788BB420CD34088834209D88888A04236
:109F600006D3A84204D8C888904201D3B04201D990
:109F70000020F0BD0120F0BD0021425C0AB10120AB
:109F80007047491C1029F8D300207047800701D082
:109F900000207047012070470A4810B5807860B1F2
:109FA000002401E0022C06D02046FEF79FF8641C36
:109FB000042CF7D310BD0324F6E7BDE81040FEF7EC
:109FC000B9B800002822002003480179C90702D04F
:109FD0000078FEF7EBB97047282200201721018096
:109FE00041800021017141711B218171C171704754
:109FF0002DE9FE4F2B4D984691460F00824601D029
:10A0000000260DE0684600F0D5FB6A460021504668
:10A0100003F001F82878009E10B99DF8090098B166
:10A020004A463146504604F08BFE04460146002263
:10A030005046FFF73FF90D2C32D008DC84B3082CD2
:10A040002ED00B2C0BD12BE00520BDE8FE8F112C60
:10A0500010D0862C1AD0A4F54050023820D0032509
:10A06000B8F1000F04D0324621465046FEF7AAFE52
:10A070002846EAE73A4629795046FDF77DFB4A46ED
:10A08000E9785046FDF778FB0025E9E73A4629795B
:10A090005046FDF771FB4A46E9785046FDF76CFBE8
:10A0A0002546DDE7882200202DE9F041204F0E46AD
:10A0B000154604463978FDF747FB002835D0204681
:10A0C00002F0A0FF50B32046FFF7BCFD80462046BB
:10A0D000B978FDF739FB08B1012700E002272046D7
:10A0E00003F038FA0028404602D0FFF797FD0DE054
:10A0F000A8F57F41FF3909D0072103F0A9F8010035
:10A1000004D0052902D0204604F080FB2B463246BD
:10A1100039462046BDE8F041FEF7F2BB2A463146FB
:10A120002046BDE8F041FEF761BDBDE8F0810000CA
:10A130008022002070B5094D0646E978FDF704FB42
:10A14000044629793046FDF7FFFA0146224630469B
:10A15000BDE870400123FFF74BBF000088220020BC
:10A160002DE9F047394E002780463D46DFF8E09064
:10A17000D6F804A057E003D00446D0F81C8035E0A0
:10A1800099F8002002EB4201521CD2B289F800205B
:10A1900009EBC10199F80230091D9A4201D189F8F1
:10A1A000005048680A780446012A12D0022A02D0D8
:10A1B000032A3BD108E004F06BFF00B101272574AE
:10A1C00034E00574C06900E070680028F9D170605F
:10A1D0002CE0207C50BB88686060C868A06008697B
:10A1E000E0604869A061F07800B165606268B168BC
:10A1F000184B501A20F07F40984202D2A1680844C0
:10A2000006E0881AA16820F07F40814202D9081A2E
:10A21000206000E0256065600120A5602074204674
:10A22000E56104F017FFB8F10000A4D199F800101F
:10A2300099F801008142A3D117B97168514502D044
:10A240000120BDE8F0870020FBE70000E8220020A5
:10A25000F4290020FFFF7F0030B585B005460024BB
:10A2600014216846FCF71BF9A5F57F40ADF80250B4
:10A27000FF3815D02846FFF7B9FA98B10B2815D04A
:10A28000112811D0A0F54051023903D001462846CB
:10A2900004F0A8FA09482246C1782846FDF76CFA6E
:10A2A00005B030BD0E2002E00124F3E70F208DF849
:10A2B00000006846FEF7C0FDECE7000048220020E1
:10A2C0000A4602498978FDF757BA00004822002063
:10A2D000F8B5054600780C46002620420FD1002034
:10A2E0008DF800006846FCF7AFFD2878204202D1C7
:10A2F0002043287001269DF80000FCF7C9FD304678
:10A30000F8BD00002DE9FF410026234800F013FBB3
:10A310002148001F074600F00EFB204C60680090AB
:10A32000A56800E000986946284004EB80000C30E6
:10A33000FFF7D2FD0028F5D101AA009901EA050333
:10A3400004EB8303491CDB6842F82030401C009179
:10A350000228F2D3019800F0030001280BD0022854
:10A3600010D10198032101EB90500099BDF80A60CB
:10A3700001EB900005E00198BDF80A60C0F383107E
:10A3800008440090384600F0D3FA08B100986060A5
:10A3900004B03046BDE8F081D0310020B82D002057
:10A3A000ACB04FF40041002001F0B2FC08B1FCF762
:10A3B00069FC01F01DFBFCF7C9FC08B1FCF762FC6D
:10A3C00001F0C4FD08B1FCF75DFC63490320FDF713
:10A3D000A3FF08B1FCF756FC69460020FDF7CEFE4E
:10A3E00008B1FCF74FFC9DF8000002287DD0002545
:10A3F00001F09CFF08B1FCF745FC002469460120F0
:10A40000009401F021FE08B1FCF73CFC684601F025
:10A410009FFE08B1FCF736FC03F0A2F99DF8080096
:10A420004EA120F00F00401C20F0F00010308DF8FD
:10A430000800112202A87CDF08B1FCF723FC00947D
:10A440005020ADF80000A0200194ADF80200ADF856
:10A4500004404FF4C870ADF8060068467ADF08B1D2
:10A46000FCF710FC0021424800F0FBFA08B1FCF7B1
:10A4700009FCAC216846FCF712F802208DF80000B8
:10A4800001208DF802000621ADF810008DF87C0047
:10A490008DF803104FF4967036492290059144F2DE
:10A4A0005060239034482990314869462030FCF7A9
:10A4B000D9FE08B1FCF7E6FB2D4801212030FCF75E
:10A4C000CEFE2E4801A9CDE900402948143000F005
:10A4D00088FB08B1FCF7D6FBFDF7A8F908B1FCF73B
:10A4E000D1FB27480090684600E032E0FDF774FA9F
:10A4F00008B1FCF7C7FB1C216846FBF7D0FF4FF4FF
:10A500002030CDE900404FF4702002901D480590A6
:10A5100003261D488DF80C600690ADF80E408DF8AE
:10A5200010406846FDF798F808B1FCF7ABFB1748F8
:10A5300017A1008806EB004001F078FB2846FCF7E5
:10A54000BFFA00BF01F062FA0028FBD101F026FD3E
:10A55000F8E701254CE70000718202004E6F72643B
:10A5600069635F427574746F6E6C6573730000008D
:10A57000342400202222002009CC020031C0020035
:10A58000FD7B02002DCC0200B388020024240020B1
:10A59000427574746F6E6C65737320444655204128
:10A5A00070706C69636174696F6E2073746172742A
:10A5B00065642E0070B5144682880E4605462088D4
:10A5C000111D0144921C994201D8FE2A01D90C2088
:10A5D00070BD521C32542088FF21401C80B2208064
:10A5E00031542088401C80B220808119288804F0D2
:10A5F00067FF2188084480B22080AA8842B1A968F8
:10A6000041B13044FBF732FF2088A98808442080FC
:10A61000002070BD072070BD2DE9F047C7880446B3
:10A62000181D16468946B0FBF7F1B0FBF7F207FBA1
:10A6300012009A193A44D21CB2FBF7F2DDF820A0BE
:10A6400001E02468491E0029FBD13D1A8846B54225
:10A6500016D818E0BAF1000F05D0211809EB080050
:10A660002A46091D04E0204409EB08012A46001D82
:10A67000FBF7FCFE00202468761BA844B74201D9F2
:10A68000354600E03D46002EE4D1BDE8F0870000ED
:10A6900030B5024659B101F067FB0021074C09E0D3
:10A6A00004EB810315685B88AB4202D11160002086
:10A6B00030BD491C8142F3D3052030BDF423002076
:10A6C000F8B50F46017814460546012901D168788E
:10A6D00030B12088821C9A422DD8012902D006E090
:10A6E0000720F8BD69780144891C994223D8181ABB
:10A6F000801E86B2ADF800602188B81C0844694607
:10A700007DDF0028EDD12878022805D1BDF80010A2
:10A71000B14201D809210AE00821012805D1687851
:10A72000B04202D8ADF8000001E0ADF80060BDF81D
:10A730000000FE2801D90C20F8BD2288401CB85426
:10A740002088401C80B2208039542088401C208002
:10A75000BDF80010084420800020F8BD70B5054603
:10A760000C004FF0FF0020D04FF6FF76B5421CD012
:10A770000E48012241782846FCF7FEFF2846FEF7E6
:10A7800099FFFF2803D1FEF7B1FFFF280DD0084B3A
:10A7900000EB400203EB82014D8023F82260226827
:10A7A0004A60A2880A81A2798A7270BD5A2200206A
:10A7B00040260020034A00219268C0E90021816000
:10A7C000704700008822002070B54FF6FF750E46D6
:10A7D000A84201D1002000E0401C84B208E02146DC
:10A7E000304603F088F908B1204670BD641CA4B25D
:10A7F000FF2CF4D9284670BD10B5FBF756FD08B103
:10A80000002010BD112010BD10B531B1B2FBF3F422
:10A8100003FB14241CB1092010BD0E2010BD0160E3
:10A820000021416081608281C381084610BD70B5FE
:10A830000C460546FBF7EEFC002802D0218828686C
:10A84000084470BD10B50A8849888A4203D1FBF7D5
:10A8500023FD012010BD002010BD70B50C4605463B
:10A86000FBF7FDFC002802D061882868084470BD11
:10A8700010B50A8849888A4203D1FBF7E7FC01201A
:10A8800010BD002010BD01F01F0301229A40D243E9
:10A89000490900EB8100114600F059B80A4601F061
:10A8A0001F030121994010B552090C4600EB8200AC
:10A8B00000F05DF8204000D0012010BD2DE9F041EE
:10A8C00080460D460024481E012101EB501716E07A
:10A8D00058F82400C04390FAA0F0B0FA80F0202885
:10A8E0000CD200EB4416AE4208D231464046FFF788
:10A8F000D5FF0028ECD13046BDE8F081641CA742AA
:10A90000E6D82846F8E74A0950F8220001F01F026D
:10A9100001219140084000D00120704701F01F0341
:10A9200001229A40490900EB8100114600F029B844
:10A93000002100F017B8012100F023B8012100F038
:10A9400016B808B56A46FBF7FCFC009808BD08B5C8
:10A950006A46FBF7DCFC009808BD08B56A46FBF7C1
:10A96000F0FC08BD08B56A46FBF7D1FC08BD08B588
:10A970006A46FBF7BFFC08BD08B56A46FBF7AEFCAC
:10A9800008BD08B56A46FBF7B5FC009808BD08B5D8
:10A990006A46FBF7E3FC009808BD38B5044600257D
:10A9A0008DF800506846FCF74FFA21686268086825
:10A9B00090420ED9401E08600178A38AE26801FB2C
:10A9C0000325227A2168101AC0B20A79824200D285
:10A9D00008719DF80000FCF75BFA284638BD38B5D1
:10A9E000054600208DF800000C466846FCF72CFA5E
:10A9F000E868A98A201AB0FBF1F12A681068431CA4
:10AA0000136001709DF80000FCF742FA38BD10B5E4
:10AA100030B1017A42680368891AC9B21A6006E047
:10AA20000E2010BD03681A68541C1C601170491E6A
:10AA3000C9B2F7D2006800210171084610BDC208F2
:10AA400000F007030120895C98400840704710B56A
:10AA5000C20800F00703885C01249C40204388540E
:10AA600010BD10B560B10161172120F8021B20F85C
:10AA7000021B1B2100F8021BFFF7B0FA002010BDDB
:10AA80000E2010BDF0B5858893B00C46002D39D14D
:10AA9000018800263E4F24293BD006DC102909D02E
:10AAA00011290CD0232958D14FE03A290BD0552930
:10AAB00053D129E00146204602F0C6F84DE0A01D22
:10AAC000FFF78CFA49E02246408934F8061F81429C
:10AAD00000D808466080172800D2172060801069CF
:10AAE00070B1607960B1D7E90001CDE90301ADF83B
:10AAF0000E506088ADF81000136903A910469847FE
:10AB00006671267113B0F0BD0146204602F0ECF8E4
:10AB100023E0011D2C2206A8FBF7A8FCBDF81800B5
:10AB2000BDF81C2004EBC0014A732269AAB1D7E921
:10AB30000423CDE90423ADF81200487B8DF81400FE
:10AB40002269204604A9904707E0017A207B8842C9
:10AB500000D201462846FDF7F5FEA07A0028D1D0A4
:10AB6000E1882846A5DF012570B11128CAD001F07F
:10AB70009FFC0246074808A1008813B005EB00407F
:10AB8000BDE8F04001F056B8A672E572BAE70000E1
:10AB900048FC0200F423002073645F626C655F6709
:10ABA000617474635F65786368616E67655F6D7417
:10ABB000755F726571756573742829207265747587
:10ABC000726E65642025732E0000000020B10278AB
:10ABD000DE2A03D0082070470E20704741800020F5
:10ABE000704760B159B10278DE2A0AD00968416025
:10ABF000DE2101704FF6FF714180002070470E206A
:10AC00007047082070477FB5054600294DD0002DBC
:10AC10004BD008780C46DE2847D1A8886188884246
:10AC200002D1204604F00CFD2888012825D00228F6
:10AC30003BD011283AD0512837D135F8040F61881C
:10AC4000884232D1A978A81C02292ED1017A042980
:10AC500003D0062901D0052927D100210091022225
:10AC60008DF8002001914FF4C07202910391ADF86C
:10AC70000420007A05280FD010E0297A2046012907
:10AC800013D1A988428891420FD10121017204B0E9
:10AC9000BDE8704004F0D4BCADF8041028886946C3
:10ACA000B0DF002801D0616888477FBDA88861882F
:10ACB0008842FAD14FF6FF7060807FBD00F180407E
:10ACC0000068002800D00120704708B500F18040DE
:10ACD000002101600068009008BD000070B54FF0D1
:10ACE00010246169104D0126491C288814D062691E
:10ACF000032101EB00400DA100F09CFF606913DF10
:10AD0000040007D0288814A106EB004000F08EFF55
:10AD1000204670BD002070BD06EB00401BA100F076
:10AD200085FF042070BD0000242400205365747446
:10AD3000696E6720766563746F72207461626C65FA
:10AD400020746F20626F6F746C6F616465723A205B
:10AD500030782530387800004661696C656420726F
:10AD6000756E6E696E672073645F736F6674646579
:10AD7000766963655F766563746F725F7461626C38
:10AD8000655F626173655F73657400004E6F20627A
:10AD90006F6F746C6F616465722077617320666F8A
:10ADA000756E640070B50C4D03210C4A288801EBC8
:10ADB00000400BA100F03EFF084813DF040008D05C
:10ADC0002888012101EB004010A100F02FFF204650
:10ADD00070BD002070BD000024240020006002002F
:10ADE00053657474696E6720766563746F7220743E
:10ADF00061626C6520746F206D61696E2061707096
:10AE00003A20307825303878000000004661696CBF
:10AE100065642072756E6E696E672073645F736F10
:10AE200066746465766963655F766563746F725F87
:10AE30007461626C655F626173655F736574000065
:10AE400070B50B4C207808B185250FE00020A0607C
:10AE500060602061E060074801F066FB054601F094
:10AE6000B1FA08B901F04AFB01202070284670BDF4
:10AE7000042900202587020038B500258DF80050F0
:10AE80006846FBF7E1FF074CE068401EE060E068C1
:10AE900010B901F059FBA5709DF80000FBF7F8FF11
:10AEA00038BD000004290020F0B505460478154897
:10AEB00089B0164640F82420124A08690832A2F1E7
:10AEC0000C0742F82400487F385520226846FBF7DB
:10AED000CDFA04942878385C48B10EB10A4A00E0F3
:10AEE00000226946281D01F0ABFD09B0F0BD0EB18E
:10AEF000064A00E00022694605F10C0001F072FCF0
:10AF0000F3E70000A82200209DF30200E9F102000F
:10AF10000FB408B50399002904D004AA00926A4628
:10AF200000F00FF801B05DF814FB10B5826804461C
:10AF3000002A05D0D4E90403216898470020A060C6
:10AF400010BD2DE9FC4791460C00804676D014F8E0
:10AF5000011B39B125290ED04046FDF74FFB207863
:10AF60000028F4D198F80C00002867D04046BDE8CE
:10AF7000FC47FFF7DABF0020012221782B291BD0E4
:10AF80002D2902D0302908D102E040F0010001E073
:10AF900040F00200641C002AEFD100252A290ED0BF
:10AFA0002178A1F130020A2A11D205EB850201EBCA
:10AFB0004205641C303DF1E740F00400EAE7D9F8AF
:10AFC00000100B1DC9F800300968641C0D4421787D
:10AFD00000232E290BD114F8011FA1F130020A2AF7
:10AFE00005D203EB830201EB4203303BF3E76C290C
:10AFF0000DD068290BD0692921D00BDC252918D068
:10B00000582931D063290ED0642915D117E014F8DE
:10B01000011FECE7702969D0732932D075291BD044
:10B02000782909D120E0D9F80000011DC9F80010E5
:10B0300001784046FDF7E2FA641C90E76CE0D9F82D
:10B0400000100A1DC9F800200968CDE900500A2245
:10B050004046FEF7ADFEEFE7D9F800100A1DC9F82B
:10B06000002009680A2206E0D9F800100A1DC9F874
:10B07000002009681022CDE90050404604F036FA5D
:10B08000DAE7D9F8001000270A1DC9F800200E6879
:10B09000C00705D112E04046761C7F1CFDF7AEFAD2
:10B0A00031780029F7D104E0202140466D1EFDF7DC
:10B0B000A5FABD42C0D9002DF6D1BDE74EB130464C
:10B0C000FBF7F8F9074604E0202140466D1EFDF726
:10B0D00095FABD4206D9002DF6D103E04046761C14
:10B0E000FDF78CFA31780029F8D1A5E7D9F80000EE
:10B0F000011DC9F80010056830214046FDF77EFAB1
:10B1000078214046FDF77AFA08200021CDE90001B8
:10B11000034610222946B0E7BDE8FC872DE9F84F29
:10B120002B4E04009A4630884FF00103154689469D
:10B1300003EB004024D0216800292BD0002D32D011
:10B14000626849464FF010071268A2F1010C1CEA30
:10B15000090F11D198466A432046FBF78AFC002864
:10B160002AD0206853462A46066901B0494620463F
:10B17000B446BDE8F04F6047164B17A2009721E098
:10B180000E210091134B1EA21FA100F062FD0E20A4
:10B19000BDE8F88F082100910E4B26A21AA100F0FD
:10B1A00058FD0820F4E7092100910A4B24A216A1BA
:10B1B00000F04FFD0920EBE700973188054B214A4D
:10B1C00008EB014010A100F044FD1020E0E7000072
:10B1D000142400209BFD0200616464725F69735F48
:10B1E000706167655F616C69676E656428705F6632
:10B1F000732C20706167655F6164647229000000D0
:10B20000705F667300000000257320636865636BE0
:10B21000206661696C656420696E20257328292089
:10B22000776974682076616C756520307825782E92
:10B2300000000000705F66732D3E705F61706900F2
:10B240006C656E000002030038B503000F484FF034
:10B2500001054FF00E04008805EB004009D061B1F4
:10B2600019600C6801B0A446BDE83040114618468C
:10B270006047074B07A2009402E0054B07A2009429
:10B2800008A100F0E6FC0E2038BD000014240020C8
:10B2900050FD0200705F667300000000705F617017
:10B2A00069000000257320636865636B206661692F
:10B2B0006C656420696E202573282920776974687D
:10B2C0002076616C756520307825782E00000000AE
:10B2D0002DE9F04128B1016819B1C969BDE8F04113
:10B2E00008470D4D0D480024461B14270DE000BFF4
:10B2F00004EB840005EB8000016829B1C969884727
:10B3000010B10120BDE8F081641CB6FBF7F0A0424B
:10B31000EED80020F6E70000E0230020F423002010
:10B32000044801214174007A08B1002070470120CF
:10B3300070470000782C0020012801D0032808D194
:10B340000449002201284A7400D00020087402F049
:10B350007BBE7047782C002070B50246022801D0D1
:10B36000032A45D1234C207A002841D0012833D02C
:10B37000022831D120480023022A006802D0032A83
:10B380002AD11BE0E360017911B1012924D10DE03C
:10B39000D0E90565711B4FF48056B14200D33146A8
:10B3A000294481614569A9420ED015E00169491C13
:10B3B0000161426991420FD1237213E0E168491C97
:10B3C000E160082908D9E3602372022A0AD00D211E
:10B3D000FDF7CEFC02F0DEFD607C28B1BDE87040D8
:10B3E00000F0F6BF0021F3E7BDE8704002F02CBE8C
:10B3F00070BD0000782C0020542300202DE9F84F68
:10B400003A4D04008B4628884FF00106DDF828A04D
:10B41000984691464FF00E0106EB00401AD0B9F164
:10B42000000F1BD02168002920D00921B8F1000F9E
:10B4300025D062685368B8FBF3F703FB1782002A34
:10B4400021D02B4B2BA2009135A100F002FC09204A
:10B45000BDE8F88F264B3DA2009102E0244B3DA2AF
:10B4600000912FA100F0F5FB0E20F1E708210091DB
:10B470001F4B3AA22AA100F0ECFB0820E8E71C4B86
:10B4800039A20091E0E75846FBF7EDFA102798B192
:10B490004846FBF7E8FAB0B1424659462046FBF76A
:10B4A000E8FAB8B1CDF800A0206843464A46C5681E
:10B4B00059462046A847CBE7009728880C4B06EB57
:10B4C00000402AA20CE000972888094B06EB0040B8
:10B4D0002CA205E000972888054B06EB004032A21D
:10B4E0000FA100F0B6FB1020B2E7000014240020EA
:10B4F00088FD020021286C656E202520705F667330
:10B500002D3E705F666C6173685F696E666F2D3E7D
:10B5100070726F6772616D5F756E697429000000EB
:10B52000257320636865636B206661696C656420C0
:10B53000696E202573282920776974682076616CEC
:10B54000756520307825782E00000000705F6673E6
:10B5500000000000705F737263000000705F66732C
:10B560002D3E705F617069006C656E00616464728D
:10B570005F69735F616C69676E6564333228646507
:10B5800073742900616464725F69735F616C6967D9
:10B590006E65643332282875696E7433325F74299E
:10B5A000705F737263290000616464725F69735F26
:10B5B00077697468696E5F626F756E647328705F17
:10B5C00066732C20646573742C206C656E290000F2
:10B5D0002DE9FF411C46DDE90A7815460E4668460E
:10B5E00000F0AAF846EA450141EA840141EA07224F
:10B5F00042EA0841009A00EB8200C0F80017BDE85B
:10B60000FF812DE9FF411C46DDE90A7815460E460B
:10B61000684600F09FF846EA450141EA840141EAA4
:10B62000072242EA0841009A00EB8200C0F80017A6
:10B63000BDE8FF812DE9FF411C46DDE90A7815468A
:10B640000E46684600F094F846EA450141EA840156
:10B6500041EA072242EA0841009A00EB8200C0F862
:10B660000017BDE8FF812DE9FF411C46DDE90A789E
:10B6700015460E46684600F089F846EA450141EA5B
:10B68000840141EA072242EA0841009A00EB820065
:10B69000C0F80017BDE8FF811CB5002100910B46E2
:10B6A00001220191FFF7C6FF1CBD1CB500210091CE
:10B6B0000B4601220191FFF7D6FF1CBD1CB50022ED
:10B6C0000B46009211460192FFF7B4FF1CBD1CB55A
:10B6D00000220B46009211460192FFF7C4FF1CBDE9
:10B6E0001CB5002100910B46012201911146FFF784
:10B6F000A1FF1CBD1CB5002100910B460122019148
:10B700001146FFF7B0FF1CBD13B50C46684600F0AC
:10B7100021F8009900EB8101D1F8002722F4403292
:10B72000C1F80027009900EB8100D0F8001741EA2A
:10B730000441C0F800171CBD0168202902D24FF057
:10B74000A040704701F01F010160014870470000F0
:10B75000000300500168202902D24FF0A04070473A
:10B7600001F01F0101600148704700000003005014
:10B770000168202902D24FF0A040704701F01F015C
:10B780000160014870470000000300500168202953
:10B7900002D24FF0A040704701F01F010160014844
:10B7A000704700000003005001B56846FFF7D2FF64
:10B7B000D0F810050099C84000F0010008BD01B59F
:10B7C0006846FFF7D5FF009A01219140C0F808159F
:10B7D00008BD01B56846FFF7D9FF009A01219140E5
:10B7E000C0F8081508BD38B501240090684631B18D
:10B7F000FFF7A2FF00998C40C0F8084538BDFFF75D
:10B800009BFF00998C40C0F80C4538BD1CB5094C15
:10B810000144D4E90034CDE900346C4606E000BFB1
:10B8200054F82030D3F81035401C08C28142F7D8B4
:10B830001CBD000000FD0200034908B508440021BA
:10B8400001600068009008BD006000400249405857
:10B85000012800D0002070470060004030B5124B36
:10B8600001460020D3F81044224609E0157A8542AB
:10B8700005D1401C0A28F7DB4FF0FF3030BD52687D
:10B88000002AF3D1421CF9D00872D3F810242AB14F
:10B8900052684A60D3F81024516030BD0022C3F8CA
:10B8A00010144A6030BD0000B82D0020F0B595B0EE
:10B8B0001C4615460F4608461A9E00F025FB182127
:10B8C00009A8FAF7ECFD0E96CDE9095400230822E9
:10B8D00003A9384600F02DFB05980690BDF810002E
:10B8E000ADF81C00BDF81200ADF81E0000208DF868
:10B8F00021000398082600F00300012802D0022846
:10B9000018D032E003983346850AC0F3C2008DF8A0
:10B91000200003980FA9C0F38314A200384600F05A
:10B9200008FB09A8009006AB22460FA9284600F0A4
:10B9300047FA1AE00398840DC0F3C2008DF8200086
:10B94000082C01D2254600E0082533462A460FA9D7
:10B95000384600F0EEFA2E44641B09AB06AA2946CD
:10B960000FA800F07FF9002CEAD1384600F0D2FA97
:10B9700015B0F0BD7047012003F054BC084810B565
:10B980000178084A515C19B1001D01F0E5F802E0A8
:10B990000C3000F0F3FFBDE81040002003F042BC83
:10B9A00068230020A422002008B5034A0092402307
:10B9B000024AFFF77BFF08BD35E80200B82C0020E3
:10B9C0000A4A012902EBC00007D0022907D0032947
:10B9D00007D0042907D000207047022070470420B8
:10B9E000704700797047407970470000FC080300F9
:10B9F00010B5FFF7C0FF04210348FFF72FFF0249EE
:10BA00000120487210BD00007C2300202DE9F04F7A
:10BA10008DB0FCF703FE18B100200DB0BDE8F08F2B
:10BA20007A4C4FF0000BC4F818B4BFF34F8F606826
:10BA30000290A568D846284004EB800008E0216801
:10BA40000298814201D86160E6E7284004EB80005B
:10BA50000C3002A9FEF740FA0028F0D105AA02999D
:10BA600001EA050304EB8303491CDB6842F820303C
:10BA7000401C02910228F2D3059800F0030002282E
:10BA800002D001284ED0A9E005985022810D8946A8
:10BA9000B2EB905F00D850210E4666F39F500590A0
:10BAA00008315B4800F0E7F9070079D000F02CFA84
:10BAB0004346082205A9384600F041FA029908F1E8
:10BAC000080A2940681A8000001D864223D94F4D7C
:10BAD0000C3530B1C2B204EB8101301A90460C3102
:10BAE00004E02946F2B2002590462846C6B25346E5
:10BAF000384600F024FA0AEB08032DB132462946F5
:10BB00004FEA070000F01BFA029909F1030001EB6C
:10BB1000900002903BE004EB8101534632463846E8
:10BB20000C31EFE70598C0F38310062800D30620F8
:10BB3000059960F38911C1F38310801C0591810080
:10BB4000334800F098F9070048D000F0DDF943468B
:10BB5000082205A9384600F0F2F908F10808002685
:10BB60000FE00298434600EA0501401C04EB810106
:10BB70000290042238460C3100F0E1F908F1040883
:10BB8000761C0598C0F38310B042EAD847B1D4F8C8
:10BB90001054D4F8180468B1384600F0BBF92FE00F
:10BBA0001CE0687A012804D12A68284639461268C0
:10BBB00090476D68002DF4D1384600F0ABF98DF850
:10BBC00000B06846FBF740F9D4F8180408B90298A9
:10BBD00060609DF80000FBF75BF911E0D4F81044B9
:10BBE00004E021682046896888476468002CF8D101
:10BBF00008480221008801EB004007A100F016F878
:10BC0000FCF70CFD80F0010007E70000B82D0020D4
:10BC10007C090300242400204261636B656E647319
:10BC200020666C75736865640000000000231A4686
:10BC300003F08AB908B5012300926A4603F084F93B
:10BC400008BD1CB5CDE9002302236A4603F07CF948
:10BC50001CBD3EB5069C8DE81C0003236A4603F01C
:10BC600073F93EBD2DE9F0470E4680461C469246CC
:10BC700008293ED894F80C900020207319461046ED
:10BC800002F01AF90025B54206D218F805201AA1CB
:10BC90002046FFF73DF903E019A12046FFF738F9E8
:10BCA0006D1C082DEFD317A12046FFF731F90025B1
:10BCB000B54210D218F80570FAF7D4FB0068C05DE1
:10BCC00010F03E0F01D03A4600E02E220EA1204691
:10BCD000FFF71EF903E00DA12046FFF719F96D1CCF
:10BCE000082DE5D301222146504602F0C7F884F81A
:10BCF0000C90BDE8F087000020253032780000006D
:10BD0000202020007C0000002563000020000000AF
:10BD1000104810B5FF218160002101604160C0F82A
:10BD20001814C0F8141480F820140B4800F0F0F830
:10BD300000280DD109480A490A4B401AC1080020C1
:10BD400003E000BF23F82000401C8842FAD3002003
:10BD500010BD0000B82D00207C0903007C09030001
:10BD6000FC080300F423002002480349401AC008DD
:10BD7000704700007C090300FC08030013B5684607
:10BD8000FEF786FC08B100201CBD0248009950F85F
:10BD900031001CBDFC08030070B508480125D0F82F
:10BDA000104480F8205405E06572216820464968F7
:10BDB00088476468002CF7D170BD0000B82D0020C2
:10BDC0002DE9FF4781460C9D00200C462F7B2873F0
:10BDD000984616462946184602F06EF8072E42D2BB
:10BDE000DFE806F004090F161F2A360049462846E8
:10BDF000FFF78EF837E0494628462268FFF788F8B3
:10BE000031E0D4E9002349462846FFF781F82AE0CB
:10BE1000A0680090D4E9002349462846FFF778F847
:10BE200021E0D4E90201CDE90001D4E9002349462B
:10BE30002846FFF76DF816E004F1080007C88DE802
:10BE40000700D4E9002349462846FFF761F80AE0D5
:10BE500004F108000FC88DE80F00D4E9002349461B
:10BE60002846FFF755F800222946404602F006F81A
:10BE70002F73BDE8FF872DE9F041858A80462D1F8D
:10BE80004819C01CB0FBF5F0C6B24046FEF785FD70
:10BE9000041E19D00020207101206071E580002768
:10BEA0002546761EC4F800800BE04046FEF775FD7F
:10BEB00060B16179491C6171286005467F1CC0F83A
:10BEC0000080B742F1D32046BDE8F081204600F063
:10BED00002F80020F8E72DE9F041457901466B1E94
:10BEE000002201E00968521C9A42FBD30F68014608
:10BEF000002605E038460C68FEF771FD2146761CE9
:10BF0000AE42F7D3BDE8F0810121001DFEF719BD57
:10BF1000FEF77DBD10B504460121001DFEF737FD7B
:10BF200010F0FF0F04D12046BDE81040FFF7D3BF4B
:10BF300010BD38B501240094FEF76EFB38BD38B54E
:10BF400000240094FEF768FB38BD00000F4910B5CF
:10BF500000204870091D0860BFF35F8F0C490D4831
:10BF600000F062FA0A480C4A0121001FFAF7DCFED1
:10BF7000002809D106480022001F4FF40041006844
:10BF8000BDE81040FAF70CBF10BD00005C23002094
:10BF9000FCFD0200AC2C00201DC0020008B50020F2
:10BFA0008DF800006846FAF74FFFF1EE100A20F016
:10BFB0009F00E1EE100ABFF35F8F08494020C1F8EF
:10BFC00080029DF80000FAF763FF00F0FBF908B16A
:10BFD00041DF08BD20BF40BF20BF08BD04E000E036
:10BFE00070B504460C480121FEF7C6FCBFF35F8F15
:10BFF0000025002809D10120074E042C08D0311F4C
:10C000004A781AB1BFF35F8F356070BD0C7048700D
:10C0100002F0E6FCF6E700006023002003484078C9
:10C02000002802D00420FFF7DBBF70475C2300200C
:10C03000FAF728BE20B10349096801600020704763
:10C040000E207047E8FF0200FEB502460E46084685
:10C05000FFF7F0FF00286ED100250095019501241F
:10C0600006208DF80020ADF8040002958DF80240FE
:10C0700069462020326869DF2F4F48B100F018FA76
:10C080003988024604EB01432C491846FFF7D2FDDC
:10C0900000958DF801408DF80250019502958DF8BC
:10C0A000035069464020326869DF40B100F000FA71
:10C0B00002463888224904EB0040FFF7BBFD00959B
:10C0C000019502958DF8004069460120326869DFCC
:10C0D00048B100F0EDF93988024604EB01431949F3
:10C0E0001846FFF7A7FD4FF4B06000900195029548
:10C0F0006946A120326869DF48B100F0D9F9398872
:10C10000024604EB014310491846FFF793FD0095E2
:10C11000019502958DF800406946A020326869DFDC
:10C1200040B100F0C5F902463888084904EB0040E8
:10C13000FFF780FD0020FEBD2C240020980703009F
:10C14000E0070300F806030044070300A406030009
:10C150002DE9F0410446D0F8008060DF2168194DD8
:10C16000074641451CD92888022606EB004016A147
:10C17000FFF75CFD2888424606EB00401EA12368BD
:10C18000FFF75FFDF006D0F80C012168800200F196
:10C190000050421A288825A106EB0040FFF74AFD0F
:10C1A000012467B1384600F083F9024628882AA1A5
:10C1B00004EB0040FFF73EFD3846BDE8F0812E4815
:10C1C0000470F9E72C240020496E73756666696374
:10C1D00069656E742052414D20616C6C6F636174AF
:10C1E000656420666F722074686520536F667444BE
:10C1F00065766963652E00004368616E676520742B
:10C2000068652052414D207374617274206C6F63B5
:10C210006174696F6E2066726F6D203078257820AA
:10C22000746F20307825782E000000004D61786909
:10C230006D756D2052414D2073697A6520666F726D
:10C24000206170706C69636174696F6E206973201E
:10C25000307825782E00000073645F626C655F653E
:10C260006E61626C6528292072657475726E6564F2
:10C270002025732E00000000DB23002030B5144879
:10C2800091B00078002820D05FF03405ADF8405020
:10C2900010A903A861DF30B1052816D011B0BDE8A0
:10C2A0003040FAF7EFBC03AC0A49684600F0BCF82E
:10C2B00007E000BFD0E9002120469047684600F023
:10C2C000CAF802980028E1D0F4E711B030BD0000B0
:10C2D000DB230020ECFF0200F8B5134C2078C0B13E
:10C2E0000120A07002F022F9112814D0022002F0DF
:10C2F00035F900258DF800506846FAF7A5FD11DFE5
:10C30000064625709DF80000FAF7C2FD2EB13046B2
:10C31000F8BD0820F8BD0020F8BDA57002F0CCFDE6
:10C32000032002F01BF9F6E7D82300207CB5194C56
:10C33000207808B108207CBD0120A070002002F008
:10C34000F5F8112819D0002002F008F9124800264B
:10C35000006801908DF800606846FAF775FD0F4996
:10C3600001A810DF05000AD0002020709DF8000011
:10C37000FAF78EFD2DB128467CBD00207CBD012042
:10C38000F3E7A670667002F0B3FD012002F0E6F854
:10C39000F3E70000D823002080FF0200096C0200B0
:10C3A0000EB50749684600F03FF805E0D0E90010F7
:10C3B0008847684600F04FF802980028F6D10EBD75
:10C3C0009CFF02000148007870470000D82300203D
:10C3D0000548817819B1007818B1FFF77DBF0820B2
:10C3E0007047FFF7A3BF0000D82300201FB56846A1
:10C3F0004BDF30B1052814D004B0BDE81040FAF787
:10C4000041BC084901A800F00FF806E0D0E900217E
:10C410000098904701A800F01EF803980028E6D085
:10C42000F4E71FBD08000300016009684160AFF335
:10C43000008010B5D0E900215368994201D1002154
:10C4400004E0D1E90034A34202D01946816010BD56
:10C4500008314160F0E7816800290BD002689268DA
:10C460000A44826041684B689A4203D108314160B6
:10C47000FFF7DFBF704700000C4A10B502F5947358
:10C480000EE0991AC91001EBD171491002EBC101FC
:10C490000C68844201D90B4602E005D201F1080282
:10C4A0009A42EED3002010BD486810BD1CFE020069
:10C4B00000B5FFF7E1FF002800D1014800BD0000F2
:10C4C00008FE02004058002800D00120704708B53F
:10C4D000002242504058009008BDD0F804030840A4
:10C4E00000D0012070474058002800D0012070473C
:10C4F00008B5002242504058009008BD0848006826
:10C50000012110F0010F08D14FF0E020E02280F867
:10C510000024C0F88012C0F8001102480160704782
:10C5200000E100E0180500400649024600200B79B2
:10C530000BB1852070470A6001220A7100224A71FE
:10C5400070470000B8220020044901200860044818
:10C550000168C1F300410029FAD170470C00004086
:10C5600018040040002802D00149800108477047A4
:10C5700021FD02002DE9F0410E46804601F032F91E
:10C58000204D0028404616D0FCF794F8284490F837
:10C5900058008009032802D001280AD003E0404651
:10C5A000FFF702F928B103214046BDE8F041FFF74B
:10C5B000ABB80221F8E701F021F9002820D040466D
:10C5C000FCF778F80446104F4FF4807007EB8401B5
:10C5D00000EB8400D1F8102580B242F00102C1F8CE
:10C5E0001025FFF729F9002E0AD04046FCF762F823
:10C5F00055F82000002803D00120A040C7F804030C
:10C60000BDE8F08118290020006000402DE9FC41C0
:10C61000DFF8C080044608EB0400002790F93000E2
:10C620001346C0170E46401C01D008274FE0B078D3
:10C630001946C0F340022046FCF718F80546401C96
:10C6400044D0B07841071CD4C0070DD06846009490
:10C65000FFF780F8009900EB8100D0F8001721F077
:10C660000201C0F8001707E000217378204600910E
:10C670000A460191FEF7C5FF164920466431FEF7D0
:10C68000E6F9B078800718D51348317800EB8500BB
:10C69000D0F81025114B1A40C0F810254FF47C52E9
:10C6A0004FF4403302EA042203EA01410A43D0F87E
:10C6B00010150A43C0F8102509E008EB0500327890
:10C6C00010F8581F41EA8211017000E00427384633
:10C6D000BDE8FC811829002000600040FFC0FCFF7D
:10C6E00010B5FFF761F8002800D0012010BD000050
:10C6F00070B5194D95F86A0008B1082070BD00208A
:10C70000411E2A18401CC0B282F830103028F8D3DD
:10C7100000242046FBF79CFF641CE4B20C2CF8D3E9
:10C720000D490024E0204C66A1F868400B4981F8CF
:10C73000000401264020891FC1F88002C1F80001D1
:10C740004FF4BE70FFF778F80549F007C1F804030D
:10C7500085F86A60204670BD1829002006E000E0D8
:10C7600000600040034890F86A00002800D00120D3
:10C7700070470000182900200121B1EB507F01D142
:10C78000012070470020704738B50D4601F0E0FBEE
:10C79000040014D000208DF800006846FAF754FB1E
:10C7A000207928B19DF80000FAF772FB112038BDFE
:10C7B0000120256020719DF80000FAF769FB002038
:10C7C00038BD10B501F0C4FB002802D00021016083
:10C7D000017110BD0149024802F04CBD84290020BE
:10C7E000002000402DE9F0410546007916460F462D
:10C7F00000EB40012D4A01EBC00102EB810494F8EB
:10C800002A1011B10820BDE8F081294951F8201003
:10C810002868FFF7B9FF08B11120F4E73946284628
:10C82000FAF750FB66603869206030004FF001066F
:10C830002FD03F7F4FF48E712868FFF748FE4FF4EA
:10C84000A2712868FFF743FE28681A49C0F804134C
:10C8500028684FEA4711000B40B2002806DA00F0C2
:10C860000F0000F1E02080F8141D03E000F1E0204B
:10C8700080F800142868000B40B200F01F0206FA8E
:10C8800002F14009800000F1E020C0F88012C0F8F9
:10C89000001128680421C0F800150020A061E061A3
:10C8A00084F8290044F8140FA675ACE78429002009
:10C8B00008FD0200800002002DE9F04705460079DE
:10C8C0000B4600EB400101EBC000234901EB800463
:10C8D000284600F043F810B11120BDE8F0874FF072
:10C8E0000008C4F82080A360626184F828804FF4B7
:10C8F0008E76474631462868FFF7E9FD28684FF0F5
:10C900000109C0F808902146286802F04FFC6068D1
:10C9100000BBD5F800A00EE094F8280008B10F275E
:10C9200016E031465046FFF7CDFD0028F4D02146F1
:10C93000504602F03BFC216A60698142F1D33146E6
:10C940002868FFF7BFFD0028F9D02868C0F80C90D0
:10C95000C4F814803846C0E784290020007900EB31
:10C96000400101EBC000044901EB80004069002850
:10C9700000D0012070470000842900202DE9F047F5
:10C98000044600794FF0000900EB400101EBC000C4
:10C99000254901EB80072068C0F80095786880B1D0
:10C9A00020682249C0F8081320680121000B40B21A
:10C9B00000F01F0291404009800000F1E020C0F823
:10C9C00080112068D0F80C25D0F81485D0F80865BF
:10C9D000D0F810554FF0FF31C0F81415C0F80C1501
:10C9E0002068C0F80815C0F81015501C02D0104679
:10C9F000FEF752FEB8F1FF3F02D04046FEF74CFE74
:10CA0000681C02D02846FEF747FE701C02D0304654
:10CA1000FEF742FE2068FFF7D4FE87F82A90C7F899
:10CA20000490BDE8F0870000842900208402020001
:10CA30000149024802F0CABCB02900200020004091
:10CA40002DE9F0410546164600790F46154A00EBE0
:10CA5000C00102EB810494F8201011B10820BDE858
:10CA6000F081114951F820102868FFF78DFE08B1B8
:10CA70001120F4E739462846FAF75FFA666038690C
:10CA800020601EB1397F2846FDF7E6F928680821A5
:10CA9000C0F800150020A061E0610121606184F808
:10CAA0002010DCE7B02900200CFD02002DE9F04742
:10CAB00004460E460079204900EBC00001EB8005DA
:10CAC00017463046FFF758FE30B1204600F036F8E2
:10CAD00020B11120BDE8F0871020FBE76F61AE6048
:10CAE0004FF49076002731462068FFF701FD4FF4A0
:10CAF000AC7841462068FFF7FBFC2068AA686969AA
:10CB0000C0F84425C0F84815206801218160686894
:10CB100078B9B14649462068FFF7E5FC064641462C
:10CB20002068FFF7E0FC0643F4D000B10F27002097
:10CB300068613846CEE70000B02900200079054939
:10CB400000EBC00001EB80004069002800D001200C
:10CB500070470000B02900202DE9F0470446007915
:10CB6000274900EBC00001EB800720684FF0000967
:10CB7000C0F80095786880B120682249C0F8081391
:10CB800020680121000B40B200F01F0291404009D3
:10CB9000800000F1E020C0F880112068D0F80C255A
:10CBA000D0F81485D0F80865D0F810554FF0FF3153
:10CBB000C0F80C15C0F814152068C0F80815C0F8A6
:10CBC0001015501C02D01046FEF76FFDB8F1FF3F64
:10CBD00002D04046FEF769FD681C02D02846FEF7E9
:10CBE00064FD701C02D03046FEF75FFD2068FFF741
:10CBF000E8FD87F82090C7F80490BDE8F0870000B2
:10CC0000B02900201003020010B550B103280CD148
:10CC10000220FBF775FB002807D0BDE81040FAF7AB
:10CC200031B8BDE8104001F019BF10BD00780028F0
:10CC300007D104483B21008876DF002801D0FAF7AD
:10CC400021B870472022002070B58D88027900EB52
:10CC5000C5042273C97BA41D012902D0022904D175
:10CC600001E0008800E040882080218860888142BF
:10CC70000FD92846A5DF0126A0B1112814D0FFF74F
:10CC800017FC02460A480BA1008806EB0040FEF79D
:10CC9000D1FFA179E079814208D92846BDE87040EA
:10CCA000FBF750BE6671F4E72671F2E770BD000035
:10CCB000F423002073645F626C655F676174746362
:10CCC0005F65786368616E67655F6D74755F7265D7
:10CCD000717565737428292072657475726E656448
:10CCE0002025732E000000007CB506468D88C8887C
:10CCF00006EBC504A41D172800D217202188814205
:10CD000000D8084660800020207121882846B5DFC1
:10CD100050B1FFF7CDFB02460E480121008801EB20
:10CD200000400DA1FEF786FF6079002810D1306920
:10CD300000280DD01449D1E90201CDE90001ADF878
:10CD400002506088ADF80400326969463046904769
:10CD50007CBD0000F423002073645F626C655F6734
:10CD6000617474735F65786368616E67655F6D7425
:10CD7000755F7265706C7928292072657475726EA2
:10CD800065642025732E000048FC02007FB51A4D13
:10CD90008188AA8891422DD110F8061F022929D135
:10CDA0004188EA88914225D1017A042922D00629B6
:10CDB00020D005291ED0841C002000900221019063
:10CDC000029003908DF80010297E19B101218DF891
:10CDD000061001E040F2FD10ADF80400A888694695
:10CDE000B0DF1128FAD0BDF80400002802D1204697
:10CDF000FAF77EFE7FBD00009C28002048B1064A5D
:10CE00000168914205D140680449401802D00128C8
:10CE100000D0032070470000DEC0ADDE02FEE10E50
:10CE20008A7D022A04D90289CB881A44D21C028145
:10CE30004289C988511AC91E418170472DE9F041C4
:10CE40000D460221904600F58056298000F1080425
:10CE5000144F1BE031462046FCF776FD40B1B8F197
:10CE6000000F02D0012288F80020022816D004E02A
:10CE7000A0687969884200D9786128886188084467
:10CE8000C01C2880608804EB80040C3431462046A6
:10CE9000FCF76DFD0028DDD1BDE8F0814FF4806026
:10CEA0002880F9E71023002008B5002100910146F1
:10CEB0000823024A0248FEF7A1FA08BD38FD020025
:10CEC000E023002008B50020009004480823044A0D
:10CED00001680448FEF792FA08BD000038230020DC
:10CEE00030FD0200E02300202DE9F05F0025DFF88F
:10CEF0000891DFF808B12C464FF00308AA462F46E8
:10CF0000D9F80C0000EB07363046FFF777FF78B30F
:10CF1000012847D0032862D100204FF4806200BF6F
:10CF200056F82010491C0ED004EB84010BEB810253
:10CF3000A8F10100566003221FFA80F80BF82120A7
:10CF4000641CA4B24BE0401C9042E9D32C48016819
:10CF500079B104EB840102200BF821000BEB810175
:10CF60004E600881254828304480641CA4B205E046
:10CF700007E00221066081804FF0010A45F00105BB
:10CF80002DE004EB840100220BF821200BEB810142
:10CF900001F110024E6030460831FFF74FFF45F0B7
:10CFA0000205CDE7BAF1000F0CD0022004EB84019A
:10CFB000134A0BF821000BEB810112684A60641CD4
:10CFC0000881A4B20E480022011D06603046FFF71A
:10CFD00035FF0B48808802280CD0082005437F1CB1
:10CFE000BFB2032F8CD3B8F1020F00D20025E8B2F4
:10CFF000BDE8F09F0420F1E7E0230020B42B0020DF
:10D000003823002001494978FAF79EBB802200208E
:10D01000002101F025BF30B585B00C4605218DF803
:10D0200000101546ADF80200FCF70CFEADF8040048
:10D030006846CDE90245FBF731FF05B030BD000081
:10D0400070B5054D06460024304655F82410884733
:10D05000641C042CF8D370BD78FC02003EB5104D62
:10D06000002400BF05EB041002F04EFC641C022CEF
:10D07000F8D30124502002210094CDE90110084981
:10D08000084BB039A02201F1A00000F0F1FB08B17B
:10D0900003203EBD0348401E847000203EBD0000BA
:10D0A000F02700206D22002000F06CB900F06CB970
:10D0B00070B504460025C168184A284602EB0013E3
:10D0C0009B688B4202D102EB001003E0401C022857
:10D0D000F4DB00202178082904D0092908D013297D
:10D0E00014D112E0617A89B980B102F01DFC0DE023
:10D0F000617A59B950B100218160817B41F0020110
:10D10000817307490120087003E001252046FFF7DD
:10D1100097FF2846BDE8704001F022B8F0270020B4
:10D120006C22002000F0E5B908B513889B0000933D
:10D130006B4600F05FF908BD002300F05BB938B51D
:10D1400005460024204609E08178284600F080F852
:10D1500010B1052800D003240098401C00906946B7
:10D16000284602F0BDFB0028EED134B9284600F075
:10D17000C4F910B1072802D00324204638BD072483
:10D18000FBE71346002200F069B900002DE9F047E3
:10D190001F0015460E46814604D0072E05D0082EE6
:10D1A00016D102E00E20BDE8F0878DB1022D0FD818
:10D1B00000F0AEF960B14FF000083146484602F089
:10D1C00075FB041E06D0207BA8420DD00F20EAE795
:10D1D0000720E8E7FF214FF6FF7002F067FB041E0F
:10D1E00006D0A0F80090A670607BFF2802D00CE06B
:10D1F0001120D8E72946154800F00CFB01462046CF
:10D200006173FF2913D04FF001082573617B0F482C
:10D2100000F04EFB02000DD0ABB23146384600F0B4
:10D2200007FAB8F1000F0ED0082E05D00BE002F07F
:10D230006BFBDDE70320B6E738886FF0050101EBF3
:10D240008000796888800020ADE70000E02700209A
:10D2500070B5002402F02AFB05000BD0686820B1ED
:10D2600000F06FF9040000D00324284602F05CFBB4
:10D27000204670BD052070BD70B515460C460729C7
:10D2800003D0082C01D0072070BD02F00FFB28B19D
:10D2900005808470BDE8704002F0C6BA052070BDFC
:10D2A0007CB50D46072903D0082D01D007207CBD91
:10D2B000002602F0FBFA040002D0606810B11CE006
:10D2C00005207CBD617B0F4800F0F2FA02004FF0B0
:10D2D0000000009001908DF8025010D0237B294669
:10D2E000684600F03DF9684602F08CFA211D684658
:10D2F00000F010F90646092801D030467CBD032015
:10D300007CBD0000E02700204FF6FF7141800149FD
:10D310000968084760FC020030B587B01748FBF782
:10D3200047FF10B1032007B030BDFBF763FE08B123
:10D330008620F8E700F0CEF9002002904CF20704B6
:10D3400003900EE0694604A8FBF7FCFE0098808875
:10D35000A0F5404085B204A8FBF7B4FE284600F0D3
:10D3600075F902AA04A92046FBF7D3FE0028E9D0EC
:10D370000349012008700020D5E70000A98E0200B3
:10D380006022002000F088B900F08CB970B586B03A
:10D3900014460E46054600F03BF940B105F5404005
:10D3A00080B20F4A6946FBF7B4FE40B902E00120A3
:10D3B00006B070BD03A96846FBF7C4FE08B10020A3
:10D3C000F6E7A57003984088208004986060039871
:10D3D0008088A0F5404030806846FBF773FEE6E7A2
:10D3E00064220020024800214160816070470000F3
:10D3F00060220020F0B587B01D46144607460E4651
:10D40000FF280AD8084600F003F930B103AA3146D4
:10D41000384600F0E5F840B902E0072007B0F0BD5B
:10D4200001A903A8FBF78EFE08B10520F6E7A67058
:10D4300001984088208045B18200286890420BD333
:10D4400002996068F9F712F801E00298606003A899
:10D45000FBF738FE0020E1E70420DFE77FB586B068
:10D460001E460D460446FF282AD8A87800F0D0F8BA
:10D4700030B304F54040ADF80000A87803AA00F5E9
:10D480004040ADF802006868019028880290A978B1
:10D49000204600F0A5F80528089813D010B108A878
:10D4A000FBF7B4FE694603A8FBF770FEB0B107288E
:10D4B0001DD0082819D00E2817D003200AB070BD3F
:10D4C0000720FBE728B108AA694603A8FBF769FE15
:10D4D000ECE7694603A8FBF760FEE7E71EB13146BB
:10D4E00003A8FBF726FE0020E8E71120E6E78620E8
:10D4F000E4E74FF6FF7000F0A9B810B5FF2801D996
:10D50000072010BD00F0A8F800F02EF8002010BD94
:10D5100000F0F4B870B504460D46807800F078F855
:10D5200058B121882846FBF759FE002804D0072867
:10D5300005D0092800D0032070BD072070BD8620CB
:10D5400070BD01B56846FBF761FE002800D00320DE
:10D5500008BD00000149C978FAF7F6B8802200201A
:10D560009BB200F065B8000070B51B4D8AB000207A
:10D57000687000904FF6FF760190304603E0204639
:10D5800000F07CF8204600F087F80446B0421DD039
:10D5900004F5404080B26A4602A9FBF7C2FD0A28A2
:10D5A000EDD004F5404080B2FBF7E4FC08280FD032
:10D5B00000280BD005461422084905A8F8F756FFA5
:10D5C000ADF8184005A80795FFF79EFE0AB070BD9C
:10D5D00001206870FAE700006022002064FC02006D
:10D5E0007CB5054616460C46084600F011F80020AA
:10D5F000009005F54045019004F54044A8B2A1B261
:10D600006B463246FBF77EFD002800D005207CBD2E
:10D6100007280BD0012809D0082807D0052805D0F5
:10D62000062803D0042801D000207047012070474D
:10D6300010B503EB83034FF6FF7404EA0313817004
:10D64000DB1C99084260018010BD00000149FBF716
:10D6500039B800001028002010B50446A0F57F401E
:10D66000FF3807D004492046FBF72CF8A04201D12F
:10D67000012010BD002010BD3028002010B5044648
:10D68000044900F089FE03492046BDE810402031DE
:10D6900000F082BE102800200149FDF795B8000077
:10D6A0003028002070B50A49FDF78EF804464FF681
:10D6B000FF7507E000F02CF838B105492046FDF76A
:10D6C00083F80446AC42F5D170BD204670BD000021
:10D6D0001028002010B508484021F8F7E0FE4FF46C
:10D6E00080742146044800F0D7F921460248BDE87D
:10D6F0001040203000F0D0B910280020FF2803D8B7
:10D700000146024800F0F7B90020704710280020B9
:10D71000FF2803D80146024800F0EDB90020704709
:10D720003028002070B500252C462146044800F022
:10D73000E2F9641CA4B20544FF2CF6D9284670BD5A
:10D740001028002010B50C46FBF7B4FFFF2804D0CA
:10D75000024900EB400021F8204010BD4026002087
:10D760001CB500F073F908B1F9F78CFA00200090AD
:10D7700001909DF8000020F07E0040F00100303064
:10D7800020F080008DF8000007208DF801001020A7
:10D790008DF802009DF8030040F003008DF80300AF
:10D7A0009DF8040040F003008DF80400684600F086
:10D7B00055FB08B1F9F766FA034800F039FB002879
:10D7C00001D0F9F75FFA1CBD11D9020000680128E9
:10D7D00005D0022803D0042801D000207047012082
:10D7E000704700000449084490F93000082801DB24
:10D7F0000120704700207047182900200449084480
:10D8000090F93000082801D20120704700207047AD
:10D81000182900202DE9F0410F46060026D0306877
:10D8200020B3706810B3FF2400251CE029467068FF
:10D8300000F039F948B1FF2C00D12C46281B401CC0
:10D84000B8420ED12046BDE8F081FF2C06D108E099
:10D850002146304600F040F8641CE4B2AC42F7D3F5
:10D86000FF246D1CEDB2B068A842DFD8FF20EAE7C4
:10D870002DE9F0410400DDE90705069E16D0A9B1A7
:10D88000A3B100FB05F7974210D8C21DB6EBD20F2B
:10D890000CD358B155B1E5602160C4E9013081B2C3
:10D8A000184600F0F9F80020BDE8F0810720FBE7FA
:10D8B00070B504000D460DD0206858B1606848B1BD
:10D8C000FF2D07D000F017F920B1E168206805FBB3
:10D8D000010070BD002070BD70B504000D4611D070
:10D8E000206800280ED0606800280BD0FF2D09D0DA
:10D8F00000F001F9002805D029466068BDE87040B5
:10D9000000F005B970BD002901D001F0CDB8704715
:10D91000F8B5044600781E4D03260E281DD2DFE818
:10D9200000F0071C0F1C1D1C24351C331C352E3524
:10D93000288818A106EB0040BDE8F840FEF776B94C
:10D940006088F9F7E3FE0246207A00902888638811
:10D9500006EB00401AA1FEF77CF9F8BD002000900C
:10D9600060886946FFF7CFFFF8BDFBF725FB082865
:10D97000FAD00028F8D0BDE8F840F9F783B9BDE83F
:10D98000F8400020F9F79CB82069F2E7A068F0E7BA
:10D9900024240020436F6E6E656374656420746F89
:10D9A00020612070726576696F75736C7920626F83
:10D9B0006E646564206465766963652E000000000E
:10D9C000436F6E6E656374696F6E20736563757205
:10D9D00065643A20726F6C653A2025642C20636F71
:10D9E0006E6E5F68616E646C653A20307825782CC5
:10D9F0002070726F6365647572653A2025642E002D
:10DA000010B50F4C2168002919D04A7E002A16D083
:10DA10000278082A02D0092A11D106E0007A0128EA
:10DA20000DD10869401E086109D1F9F71DFF0028D2
:10DA300005D020684169BDE810400220084710BDAC
:10DA4000A0220020FBF706BAFBF704BA10B5FFF7D7
:10DA500063FC88B9FFF702FB70B901F027F858B9E9
:10DA600001F042F940B9FBF7C1FD28B9FBF7A6FE6A
:10DA700010B9FCF757F808B1032010BD05484FF660
:10DA8000FF718180002181604170012101700020BF
:10DA900010BD000070220020002803D0C91DC90855
:10DAA000F8F7FDBC7047002809D001F007030122F8
:10DAB0009A40D2B200EBD1001146FCF709BC704786
:10DAC0002DE9F0410D46060013D0002401270EE099
:10DAD00004F0070007FA00F0C1B206EBD400FCF72F
:10DAE000F7FB10B12046BDE8F081641CA4B2AC4243
:10DAF000EED32846F7E740B100EBD10001F0070272
:10DB0000007801219140084000D001207047F8B50D
:10DB10000400C1F3C70501F007014FF0010000FA4E
:10DB200001F0C6B20FD0605D30420CD000208DF8FD
:10DB300000006846F9F788F9605DB04360559DF8CC
:10DB40000000F9F7A5F9F8BD2DE9F041044686B0CB
:10DB500001278088FBF7B4FF6080207800263F4DC6
:10DB6000082808D0092820D04FF6FF780A2829D0A5
:10DB70000B2853D158E0607A10B1012809D04DE04C
:10DB8000A86830B1E168814203D1AE60A088A88066
:10DB900016E06878E8B3A088A98888423ED1207A48
:10DBA00006283BD100F0C0FA38E0607A88BBA8684C
:10DBB00078B3E168814231D1AE60E868401EE86028
:10DBC000E6602BE0A878E8B14046FFF76FFA4146DF
:10DBD000404517D10846FFF767FA404512D1AE70AD
:10DBE00014216846F8F75BFC0C208DF80000ADF8B6
:10DBF0000480ADF8028000272046FBF72BF9684629
:10DC0000FBF728F9687838B1A088A988884203D141
:10DC100000E003E000F088FA002F1CD006B0204698
:10DC2000BDE8F041FBF716B9A8780028F6D0AE7031
:10DC300014216846F8F733FC0D208DF80000ADF88C
:10DC40000480ADF80280A06802902046FBF702F93C
:10DC50006846FBF7FFF806B0BDE8F08170220020AF
:10DC600008B55022ADF800200A466B46072100F0A7
:10DC700001F808BD7CB51D46164B1B7883B18AB1EF
:10DC800085B12C882346641EE61704EB967626F0B1
:10DC90000306A41B1C1BE41C9C4205D007207CBD72
:10DCA00008207CBD0E207CBD0023009301932B88AF
:10DCB0000192DB1C9B08ADF800308DF802106A461B
:10DCC000FFF732FABDF800104FF6FF7202EA810149
:10DCD00029807CBD702200200349097809B1FBF737
:10DCE0009DBF0820704700007022002010B50C4630
:10DCF0000649097829B134B1FBF7A4FF2080002040
:10DD000010BD082010BD0E2010BD000070220020A4
:10DD10002DE9FF4F2A4883B09946007892468B46FA
:10DD2000B8B14FF6FF763046FFF7C0F980460020C5
:10DD30000090244801AA062100680190CDF808D07F
:10DD40004046FFF7F1F900256C1E3746072804D03E
:10DD500017E0082007B0BDE8F08F0520FAE70020A3
:10DD60000090A84201D305464746A04201D204468E
:10DD700046464046FFF79AF9804601AA0621FFF77A
:10DD8000D3F9D8B10528EAD0A8F57F41FF3901D0F1
:10DD90000320DFE70399002001B10F80BBF1000FE2
:10DDA00001D0CBF80050BAF1000F01D0AAF8006002
:10DDB000B9F1000FCED0C9F80040CBE70098D0E70A
:10DDC0007022002088FC020070B5184E86B03078B2
:10DDD000D0B10120B0704FF6FF742046FFF766F90E
:10DDE0000546A0421DD10020B07014216846F8F706
:10DDF00056FB0C208DF80000ADF80440ADF8024051
:10DE00006846FBF727F80EE0082006B070BD00BF9B
:10DE1000FFF762FF08B10320F7E72846FFF746F94E
:10DE20000546A542F4D10020EFE700007022002053
:10DE3000084A117821B1D178032903D3042070470F
:10DE400008207047044B43F82100491CD170002082
:10DE500070470000702200205028002003490978F4
:10DE600009B100F075BE0820704700007022002044
:10DE7000002801D0FAF7EEBF7047000010B50C463D
:10DE8000017A052908D0407A38B1084808A102680B
:10DE90002046FDF73DF800E01AB106A12046FDF747
:10DEA00037F82046BDE81040FDF73FB8B423002006
:10DEB000257300000D0A000038B5C3880D460446DE
:10DEC00033B114A0009015A216A12846FDF720F842
:10DED000217A05291CD0607A48B1A088FDF770FD31
:10DEE000164951F8202016A12846FDF711F8A08800
:10DEF0000021FDF743FF03461049207A143951F8F9
:10DF0000202001B02846BDE830400EA1FDF700B842
:10DF100038BD00001B5B306D000000001B5B313B17
:10DF200033316D0025734C6F67732064726F7070AE
:10DF30006564202825642925730D0A00B423002078
:10DF4000257300003C25733E2025733A2000000015
:10DF50000349884201D10348704700207047000000
:10DF600000200040C02200200146054810B500688E
:10DF7000FCF75DFC04461C21F8F791FA204610BD21
:10DF800028FD0200014602480068FCF771BC000051
:10DF900028FD0200034802490068FCF753BC00005A
:10DFA00058230020B0FD0200F0B5254D254E85B068
:10DFB00004460027686828B9214930680831FCF711
:10DFC0004CFC686001460078072817D2DFE800F0B3
:10DFD000160408080E0E12002046FBF77BFE02E036
:10DFE000204601F02BFD040028D008E02046FAF777
:10DFF00047FDF8E72046FBF7A3F9F4E70F241421C7
:10E000006846F8F74CFAA4F5E8501D3800D1002412
:10E01000019469466868FAF761FE6846FAF798FE67
:10E0200007496F60002408313068FCF70BFC044896
:10E0300001210C30FCF7ABFC0028BBD105B0F0BDD2
:10E040001023002028FD02002DE9F041234C00257B
:10E05000234E207A012730B92248311D0068FCF791
:10E06000FCFB306038B1022020723168087928B199
:10E0700001281ED116E06560BDE8F081D1E90503F5
:10E08000C01A4FF48052904200D31046B7EB900F65
:10E0900001D2820800E001220869C96818441944C5
:10E0A00029DF03E0D1E90301084428DF58B1112832
:10E0B00012D003213068FAF75BFE25726560BDE877
:10E0C000F041FFF767BF207C0028D5D1BDE8F041C3
:10E0D00000210220FDF740B92772CDE7782C0020FF
:10E0E00054230020B0FD020010B501210448FCF7C4
:10E0F00034FC002803D1BDE81040FFF755BF10BD28
:10E100001C23002010B5074C201DFCF717FC00282D
:10E1100006D1607C002803D1BDE81040FFF794BF12
:10E1200010BD0000782C0020084910B500231A46C5
:10E13000A1F10800FFF7ECFD30B1052804D0002064
:10E1400002490C39487010BD0120F9E77C220020FB
:10E1500010B510461A46F8F789F9002010BD0000E6
:10E160002DE9F0471B4F82460026387886B00028FC
:10E1700021D00024DFF86080A14600BF08EB041521
:10E18000A87B810702D410EA0A0F1BD0012628467B
:10E1900001F04AFBB0B14FF6FF71ADF802102988CB
:10E1A000ADF80410862809D007218DF800100290E0
:10E1B0006846FEF745FF06B0BDE8F08706208DF8FB
:10E1C0000000F5E7641C022CD8D3002EF3D187F8A9
:10E1D0000090F0E76C220020F02700202DE9F047A6
:10E1E00007461E481C46154600780E4670B185B19C
:10E1F0007CB1DFF86C804FF00009A08802282BD298
:10E2000000EB800118F8210010BB19E00220BDE8E6
:10E21000F0870520FBE720681FB181883A8891428A
:10E220000ED11EB101883288914209D180682860E0
:10E23000206868600A482830008928810020E6E7C5
:10E24000A088214600F05EF80028E4D1C4F80090D0
:10E25000A088401CA080D0E70A20D8E73023002007
:10E26000B42B0020F8B505464068244F0C46002624
:10E2700048B32349CA68824225D80969814222D31A
:10E28000FBF784FEF8B12889398988421BD1D5E98A
:10E2900000018A68904216D10020A7F1280200BF31
:10E2A00000EB800302EB83035B688B4205D203F52E
:10E2B00080538B4201D9208011E0401C80B202289B
:10E2C000EED30020F8BD268000960AE00098296869
:10E2D0008068884205D100986860388928810120CB
:10E2E000F8BD2088694600F00DF80028EED120889E
:10E2F000401C80B220800228E6D3E2E7DC2B00201D
:10E30000E023002070B50E4600EB8001134800EBBF
:10E3100081004468306804F5805518B1418800EBED
:10E32000810411E0083410E029462046FBF70CFB7D
:10E3300020B1012805D0022807D10DE0012034606A
:10E3400070BD608804EB80040C3429462046FBF73E
:10E350000EFB0028E8D170BD002070BDB42B00205A
:10E3600038B50C460021009101460423074A0848AD
:10E37000FDF744F808B10E2038BD064A04EB8401CD
:10E3800002EB810101200874002038BD2CFD020041
:10E39000E0230020B42B00200A46FF2803D80146C2
:10E3A0001046FFF7B4BB704710B596B050216846D1
:10E3B000F8F775F8164C14A920688088FFF796FCCA
:10E3C000002820D1BDF85000A0F57F41FF391CD0B6
:10E3D0006946FFF745FC002815D117220D480DF1BD
:10E3E0000101F8F743F80B481C2218300DA9F8F783
:10E3F0003DF80820ADF854002068064901238088C4
:10E4000015AA3431B2DF16B010BD0F20FBE70000B3
:10E41000A0220020C82800200846704770B50126B9
:10E4200070044FF0E0210025C1F88001084C401035
:10E43000C4F84803C4F8080366602F20FEF792F87A
:10E44000A660044C2F20A560FEF78CF8A57070BD67
:10E4500000100140E822002070B5054688690C468E
:10E4600000284FF4847128460AD0FEF730F8D5F81A
:10E470001805626AE1688854606A401C606270BD79
:10E48000FEF725F8D5F8180570BD1FB501238DF8E6
:10E490000030CDE90121D0E90012684690471FBD48
:10E4A0001FB501238DF800308DF808100192D0E9D6
:10E4B0000012684690471FBD10B5044606484179D2
:10E4C0002046F9F741F9002804D12046BDE8104064
:10E4D00000F0FCB910BD00004822002038B5002132
:10E4E000012548B101280CD0032809D1FEF706F810
:10E4F000BDE83840FCF7C0BC4FF0E020C0F88051C8
:10E5000038BD8DF800106846F8F79EFC064C207860
:10E5100008B9FCF795FCE068401CE060A5709DF828
:10E520000000F8F7B5FC38BD042900203EB50446CC
:10E5300009496846FDF778FF08E000BFD0E90021EF
:10E540002046904730B16846FDF785FF02980028C5
:10E55000F4D13EBD11203EBD84FF02003EB504460D
:10E5600008496846FDF760FF07E000BFD0E90021D9
:10E57000204690476846FDF76EFF02980028F5D1C7
:10E580003EBD000090FF02002DE9FC4104460C3026
:10E5900000278046FBF766FB4FF6FF750646A8424C
:10E5A000208803D1FBF74EFB064602E03146FBF71D
:10E5B00033FB20880022012100F0C6F8AE4212D0C1
:10E5C0006A4607213046FEF7B7FD60B9019D95F810
:10E5D00044003435C00705D1414605F11200FBF770
:10E5E00006FB00B12F46002320881A46394686DFF5
:10E5F00005000BD0002320881A46314600F088F829
:10E600002088294600F002F9BDE8FC81002FFBD1EB
:10E61000002320881A46314600F07AF8208800222C
:10E6200041F20601FAF7E2FAEEE700002DE9FC41BB
:10E630001D46089C16460F46804644B16B46012293
:10E6400007213846FEF7A2FD112801D010B10320A2
:10E65000BDE8FC8150210198F7F721FF0198067071
:10E660000198E560343020600198183020610198ED
:10E67000401C60610748E061019940461131FBF799
:10E68000A3F90028E3D107213846FEF709FE052843
:10E69000DDD0DDE75C280020002835D00278910726
:10E6A00001D411062FD4C2F3021104292BD89307E9
:10E6B00003D5032901D1110625D5437881788B42F2
:10E6C00021D8072B1FD310291DD8C1784B071AD486
:10E6D0000079430717D40B0715D4030713D4D207C7
:10E6E0004FEAC17201D042B10FE062B989070AD482
:10E6F000C10708D1800706D407E0890705D4C10700
:10E7000003D1800701D4002070470120704700002A
:10E7100070B50C4605466AB1002B12D0094801229B
:10E72000C1782846F9F728F821462846BDE8704008
:10E73000FBF772BA002B04D0BDE870400846FBF727
:10E740006DBA70BD80220020F0B5174D14460F46FB
:10E750000A4685B006462978F9F70EF8002F1FD033
:10E760000CB1012200E0002269783046F9F704F884
:10E77000012C17D00022A9783046F8F7FDFF0022BF
:10E78000E9783046F8F7F8FF142208496846F7F7A9
:10E790006DFEADF802608DF808406846FAF770FB30
:10E7A00005B0F0BD0122E6E7802200209CFC0200BB
:10E7B00010B586B0044614216846F7F770FE0420B1
:10E7C0008DF80000ADF802406846FAF759FB06B034
:10E7D00010BD000002498969002900D00847704730
:10E7E000AC25002030B585B00C46054614220649FC
:10E7F0006846F7F73BFEADF8025068460294FAF718
:10E800001BFB05B030BD0000D8FB020030B585B061
:10E810000C460546142206496846F7F727FEADF870
:10E82000025068460294FAF72BFB05B030BD000099
:10E83000B0FC020070B50D4C0020D2B22070201D3B
:10E840000B4D0378EB5C1BB1001DFEF72FF902E0C6
:10E850000C30FEF731F808B1F8F714FA60780028A8
:10E8600002D021780029FAD070BD00006423002076
:10E87000A42200200348002201490079F8F730BFA4
:10E88000B9E40200482200207CB50E490E4C00225B
:10E89000D1E90001CDE900016946A088FEF771FCCD
:10E8A0004FF6FF7507E00846FEF700FCA080002247
:10E8B0006946FEF766FCA188A94201D01128F2D171
:10E8C0007CBD00002CFC02005422002070B586B0F4
:10E8D000064601250024FBF71BF8112812D005DCA1
:10E8E000F0B1062828D0082808D125E0A0F540512D
:10E8F000023907D0A1F54071FF3924D001463046D6
:10E90000FFF770FF2A46124D30462979F8F734FF99
:10E91000697906B022463046BDE87040F8F72CBF52
:10E9200014220C496846F7F7A1FDADF802600124F6
:10E930006846FAF781FAE5E700253046FBF782F9E9
:10E94000FAF72EFFDEE73046FBF786FCDAE7000039
:10E950004822002000FC02002DE9F0410746806AB1
:10E9600014468846C8B3002531E000BFB96A05EBFC
:10E97000450001EB8006B088801CFE2802D90C20DF
:10E98000BDE8F0812288401C08F802002088162289
:10E99000401C80B2208008F800202088401C80B2F3
:10E9A000208000EB0801308800F08AFD21880844AF
:10E9B00080B22080B28842B1B16871B14044F7F7AB
:10E9C00055FD2088B188084420806D1CEDB297F871
:10E9D0002C00A842CAD80020D2E7FFE70720CFE7E3
:10E9E00070B5194D194C07E0016820788847002858
:10E9F00029D01548FDF72FFDA8680028F4D1FDF7B0
:10EA0000CBF900BFFDF702F80028FBD120780328DE
:10EA10000CD002280AD0FDF7D5FC00B133DF0C4939
:10EA200001200860BFF34F8F20BFFDE7BFF34F8F7A
:10EA300008480168084A01F4E06111430160BFF32E
:10EA40004F8F00BFFDE770BDAC2C00205C23002081
:10EA5000000500400CED00E00400FA0510B50020B0
:10EA6000F9F74EFC08B1F8F70DF9F9F7A3FB08B177
:10EA7000F8F708F9FDF730FC002803D0BDE8104096
:10EA8000F8F700B910BD000010B500F0ABF805486C
:10EA9000002203494078BDE81040F8F721BE00008D
:10EAA00035A102008822002000F016B910B51148E7
:10EAB000FAF7E3FB0F48401CFAF7DFFB0D48801C18
:10EAC000FAF7DBFB0B48C01CFAF7D7FB0948001D1F
:10EAD000FAF7D3FB0748401DFAF7CFFB0548401E65
:10EAE0008179182903D00121C171002010BD0320B4
:10EAF00010BD00008922002010B50078114C0A28B2
:10EB000013D004DC082810D009281AD10DE00B28F6
:10EB10000BD0132815D100220B49A079F8F7E0FD9E
:10EB200000220A49A078F8F7DBFD00220649607947
:10EB3000F8F7D6FD6078BDE8104000220349F8F7E9
:10EB4000CFBD10BD8822002011D0020035A10200E7
:10EB500070B50B4C05004FF001060CD0FFF79CFD83
:10EB600058B1286820612879207504F11000A06050
:10EB70002670002070BD0020F9E7072070BD00005E
:10EB80008822002010B504460078052802D01228FB
:10EB900021D105E06088A168BDE8104000F060B9AF
:10EBA0000F480021806880B10D48237A103000782A
:10EBB00000F0010203B101239A4206D3627AC0F346
:10EBC000400002B10122904200D20121608801235D
:10EBD0000022FBF70DFA2046BDE81040FAF75EB9B7
:10EBE0008822002030B50446008885B014284FD014
:10EBF0000ADC11282CD0132828D134F8040FF8F798
:10EC000085FD01282FD038E0192847D01A281DD1BA
:10EC1000A088FEF7F7F9002818D1A088F8F750FD72
:10EC20000028A0884BD02A4900220978F8F7A4FDD3
:10EC300002208DF80000A088ADF8020000208DF8B9
:10EC400008008DF809006846FAF71AF905B030BDDA
:10EC5000207A3D2804D04FF48851A088002224E077
:10EC600041F23D01F9E72079C00701D0012200E01F
:10EC7000022220880121FFF767FD34F8045B14228B
:10EC800014496846F7F7F2FBADF802500294DAE750
:10EC900005B0201DBDE83040FFF776BC217A201D6D
:10ECA00041B14279008802F0030205B0BDE830406E
:10ECB000FBF7FAB905B0BDE83040F8F77BB905B00D
:10ECC0000122BDE8304041F20601F9F78FBF000094
:10ECD00080220020D8FC02000A7802490979F8F75E
:10ECE0004BBD00008022002010B51448FAF7BCFA92
:10ECF0001248401CFAF7B8FA1048801CFAF7B4FA28
:10ED00000E48C01CFAF7B0FA0C48001DFAF7ACFA2E
:10ED10000A48017818290FD0417818290CD0817839
:10ED2000182909D0C178182906D00179182903D0EB
:10ED300001214171002010BD032010BD8022002060
:10ED400070B50C460546F8F7E1FC012802D043F205
:10ED5000020070BD21004FF00000FAD028467EDF8F
:10ED600070BD00002DE9F74F8AB0924688460A9898
:10ED7000F8F7CCFC06464FF6FF7900244D462746AF
:10ED80000A98FEF7E7FB8346202101A8F7F787FBE7
:10ED9000012E01D0DEB105E02F48002201790A984A
:10EDA000F8F7EAFCB8F1000F16D098F80000C00799
:10EDB00014D00A98FAF746FF0546484516D1FEF7E3
:10EDC000B1F9054648450ED04FF0010B0CE043F277
:10EDD00002000DB0BDE8F08F852721E01F48CDF877
:10EDE00010A008901CE003246CB121E0012E0AD190
:10EDF0000A98F7F7B5FE30B90A98FFF7D9FC0A98D8
:10EE0000F7F7AEFE50B101A80090534632462946AE
:10EE10000A98FFF70BFC040002D009E0852712E0F6
:10EE2000012E10D001AB002239460A987FDF04463C
:10EE300054EA07000DD000225B4629460A98FFF7E6
:10EE400067FC2046C5E701AB424639460A987FDF9A
:10EE5000EDE70122F0E70000802200205C2800207E
:10EE60003EB505460C466846FBF7A4FC6A462146BB
:10EE70002846FEF7D0F809480099C2682846FFF7EF
:10EE800071FF0446014601222846FAF713FA21468B
:10EE90002846009AF9F796FF3EBD00008822002020
:10EEA000002805D10349012048700020F9F726BC4D
:10EEB000704700000429002010B51620F7F7AEFDBA
:10EEC00048B10A4882684FF4800152B1016821F4C8
:10EED0008001016010BDBDE8104042F20100F7F76B
:10EEE000D1BE4FF0E020C0F8801110BD002B0020F3
:10EEF00010B51620F7F792FDA0B1114890F8000464
:10EF00004009082811D280B101280ED004280CD065
:10EF10000C4882684FF480016AB1016841F48001B5
:10EF2000016010BD42F2010001E042F20200BDE8C2
:10EF30001040F7F7A7BE4FF0E020C0F8001110BD59
:10EF400016E000E0002B00202DE9F84F204D9246FE
:10EF5000894606469846012269461846AF68F9F781
:10EF600005FB58B3009800210446801C09E000BF4F
:10EF700000EA07035AF8212005EB8303401C491CD3
:10EF8000DA604145F4D34FEA164AF9F705FE4AEA3A
:10EF90000041601C384005EB80003C4005EB8402DA
:10EFA000C160D06866F3C50068F3891069F39F20DB
:10EFB00020F00300401C20F00400D06095F82004ED
:10EFC00002E000BFFCF722FD0028FBD1BDE8F88F6E
:10EFD000B82D00202DE9F84F1D4C00256846D4E9D6
:10EFE00001A6F9F7E3FD002738B30023009A616812
:10EFF0001CE0D1F800C00846944503D9ACEB0202EE
:10F000000A6015E0A2EB0C0263440760D0F80CC064
:10F01000C1698146BCF1000F08D006EB030828F057
:10F020007F48C0E9018CC9F81C5005460029E0D191
:10F0300028466160FBF794F803E02846FBF790F858
:10F0400010B15046F9F77CFBE770BDE8F88F00007F
:10F05000E82200200D4B10B5596831B102680C68E8
:10F06000A24204D8A21A0A60C161586010BD0B46C2
:10F0700003E00B46C969121B21B10C689442F8D316
:10F08000A41A0C600260C161D86110BDE8220020A2
:10F090002DE9F041144E77683D462C4603E084424A
:10F0A00004D02546E469002CF9D11BE0D4B1A54277
:10F0B0000BD1F869706040B90C49012088600021CB
:10F0C000B160F0702F20FDF74DFA2168E069E8612A
:10F0D00010B10268114401607068874202D00120BB
:10F0E000BDE8F0810020FBE7E8220020001001408D
:10F0F0007CB5064600240D468DF800406846F7F7BB
:10F10000A3FE01A800F0AEFA70B10570094946608F
:10F110009DF8040048709DF80000F7F7B9FE142030
:10F12000F7F71AFB20467CBD04249DF80000F7F792
:10F13000AFFEF7E7F42900202DE9F041194D6C6886
:10F14000002C2CD0184800270068A968B846401A3F
:10F1500020F07F462068B0420CD82146361A07447A
:10F16000E469087C20B181F8108088694969884782
:10F17000002CEFD129786878814206D1401CC0B2BA
:10F180006870022801D185F80180064869780C3042
:10F1900040F82170BDE8F0411420F7F7DDBABDE872
:10F1A000F0810000E82200200415014070B50C46F3
:10F1B00005464FF48E71FDF78AF9216AA068415C1B
:10F1C000206A401C2062C5F81C1570BD1FB50022C6
:10F1D0008DF800200291816801914261D0E900120E
:10F1E000684690471FBD00001FB50A4601788DF89C
:10F1F000001041680191017A8DF80810C0680390F1
:10F20000044850F82210083850F8222068469047E9
:10F210001FBD0000B0220020014901200870704786
:10F220006423002010B588B0044620220E496846A9
:10F23000F7F71CF906200090C01F01900290039080
:10F240004FF0EB7006900CB1084A00E000226946CE
:10F250000748FBF729FE08B1F7F714FD0448001F23
:10F26000447008B010BD000050FF020019F2020007
:10F27000682300202DE9FF470C4605464FF4007136
:10F28000FDF72BF901274FF40178002618B34FF44E
:10F29000927949462846FDF715F9E0B149462846D6
:10F2A000FDF715F9C5F8088394F8290000B96F60D7
:10F2B00002208DF80000D5F88004C5F88004039082
:10F2C000A0690290E0680190A661E661D4E90012AD
:10F2D0006846904728E004212846FDF7FEF818B359
:10F2E0004FF484712846FDF7EDF8E8B12146284631
:10F2F000FFF7B2F8616AA069884215D1E06938B1B8
:10F30000E268616AA0612069E6616662E06008E027
:10F3100094F8290000B96F60C5F80883A661E26817
:10F32000616A2046FFF7B1F84FF48E7841462846CF
:10F33000FDF7C8F878B1206A6169884202D294F872
:10F34000280020B341462846FDF7C1F8616911B194
:10F350002046FFF73BFF4FF4A27841462846FDF7D1
:10F36000B1F8002818D041462846FDF7B0F894F8C7
:10F37000290000B12F60A06900280DD0A661E268C5
:10F38000616A04B02046BDE8F047FFF77EB8214629
:10F390002846FFF70BFFDEE7BDE8FF871FB50A46EB
:10F3A00001788DF8001041680191017A8DF80810FC
:10F3B000C0680390044850F82210083850F8222002
:10F3C000684690471FBD0000B02200202DE9FF4194
:10F3D0000C464FF4927705463946FDF784F800262F
:10F3E000C0B139462846FDF783F802208DF80000A9
:10F3F000D5F88004C5F880040390D5F83C058DF855
:10F400000800E0680190A661E661D4E90012684650
:10F41000904723E04FF4887739462846FDF763F894
:10F42000E0B139462846FDF763F8D5F83C15A069E8
:10F43000884213D1E06960B1E268D5F8000220F09B
:10F440002000C5F80002E069A0612069E661E06083
:10F4500001E0A661E2682046FFF722F84FF4A277A8
:10F4600039462846FDF73FF860B139462846FDF792
:10F470003FF8A06930B1A661D5F83C152046E26896
:10F48000FFF70EF84FF4907739462846FDF72BF832
:10F49000002813D039462846FDF72AF8606900286D
:10F4A0000CD0D5F84C058DF800608DF80800A068E8
:10F4B00001906661D4E9001268469047BDE8FF817B
:10F4C0000870000A487002207047000010B514212F
:10F4D0000448F6F7E4FF04480068FBF78DF90020C4
:10F4E00010BD0000782C0020B0FD02002DE9F05F77
:10F4F0008346DDE90A4A994690460D4608460127AB
:10F5000003E000BFB0FBF8F07F1C4045FAD2B945DC
:10F5100000D94F465FEACA7012D18CB15FEA8A7097
:10F5200002D5B9F1000F01D0202607E0302605E012
:10F5300031465846641EF9F761F80CB1A742F7D37B
:10F540005FF00106B9F1010F02D9A9F1010903E049
:10F55000B5FBF6F0404502D306FB08F6F2E7DFF80C
:10F560003C9000BFB5FBF6F000FB165519F80010F3
:10F570005846F9F743F8B6FBF8F6002EF2D15FEAE9
:10F58000CA7009D0002C07D0A74205D220215846C6
:10F59000641EF9F733F8F5E7BDE8F09F40FD02007F
:10F5A0000348002201498078F8F79AB8018A0200DE
:10F5B00048220020F8B5054680B2FAF7EFFB0400B8
:10F5C00013D0154E207A0027317B88420ED2A8B284
:10F5D00004F10A0175DF28B1112806D0BDE8F84012
:10F5E000FFF7F8B8207A401C2072F8BD2772307CF3
:10F5F00038B1A8B23B2176DF18B1082801D0FFF757
:10F60000E9F871690029F0D08DF80070ADF802506A
:10F6100068468847F8BD0000AC250020417939B123
:10F6200090F8B21021B990F8B40008B101207047E9
:10F630000020704701460148FBF765B9C825002046
:10F6400030B40446007A00280AD06088002166DFC2
:10F6500028B1112802D0616830BC0847012020720F
:10F6600030BC70470A494A788B78521CD2B2934218
:10F6700000D100220B78934201D100207047027024
:10F68000487800EB400001EBC000001D704700000F
:10F69000F42900202DE9FC411646DDE90854CDE9A6
:10F6A00000541F468046022200F00CF8002807D1C3
:10F6B000CDE900543B4610223146404600F002F8A6
:10F6C000BDE8FC812DE9FC5F0026DDE90C4B994685
:10F6D00092468E4680462788354630E0D8F80400AA
:10F6E000002200EB850069460068019001A864DFF4
:10F6F000002830D19DF8000050451FD10EB10021E7
:10F7000000E00221228808441118594522D846B940
:10F71000521C90B2208009F800E02088401C208014
:10F720000126218801A801EB0902694664DF00284F
:10F7300011D120889DF80010084420806D1CB8F875
:10F740000000A842CADC56B12088C01B401E80B20F
:10F75000FF2802D90C20BDE8FC9F09F80700002013
:10F76000F9E7000010B504281DD209B1032400E018
:10F770000024F8F761FC202802D24FF0A04102E0FB
:10F780000A4900F01F0001EB8000D0F8001721F4B7
:10F790004031C0F80017D0F8001741EA0441C0F822
:10F7A0000017002010BD062010BD0000000300500F
:10F7B000002070472DE9F84F114D884681461E46BE
:10F7C00017466946DDF828A02868FBF730F80400E2
:10F7D00013D01C21F6F763FE00202071C4F80090BE
:10F7E000C4E90486C4E902A769462868FBF740F823
:10F7F000FEF788FC0020BDE8F88F0420FBE700003E
:10F80000B0FD020082780121012A0BD0062A09D01E
:10F81000072A06D0082A06D1416889880931890853
:10F8200000E01421018070471CB5044600200090C0
:10F830000190A0788DF80200617B1A48FEF738F835
:10F84000020017D0237BA1786846FDF789FE684641
:10F85000FFF7D8FF208804F1080369466268FDF7C6
:10F86000FDFD48B1072806D001210F4A112808D014
:10F8700086280FD003201CBDA17B21F00301A173BA
:10F880001CBDA07B20F0010040F00200A0731170AD
:10F8900000201CBDA37B23F0020343F00103A373EC
:10F8A00011701CBDE02700206C22002038B50546F1
:10F8B0000C46002001E00098401C00906946284654
:10F8C00000F00EF800280AD08178A142F3D1817BA4
:10F8D0008A07F0D4C907EED181680029EBD138BD81
:10F8E00010B5084B0A6809E003EB0214248884422F
:10F8F00003D103EB02100A6010BD521C022AF3D39D
:10F90000002010BDF02700204FF6FF710180FF217D
:10F9100081704173817B21F00301817300210173A8
:10F92000416081607047000070B50546002406E024
:10F93000687B2044C1B20648FDF7CEFF641C287BDB
:10F94000A042F5D82846BDE87040FFF7DDBF0000B3
:10F95000E02700202DE9FC47064636489846144625
:10F9600000780D464FF0000978B37DB32888A0F5E4
:10F970007F41FF3931D0688848B36868FAF706FBE1
:10F9800068B374B32088ADF80000678801A8FEF75B
:10F99000EBFA04002FD084F800804FF0000A84F8BE
:10F9A00016A0BDF80000A0826868206121480121EE
:10F9B0000C38FAF7C6FFE060288820816888A080AC
:10F9C000E780B8F1030F1DD020E001E003E004E080
:10F9D0000220BDE8FC870520FBE70420F9E70320AF
:10F9E000F7E7FFE72889694687B2384600F0ACF8A8
:10F9F0000028EED1CAE7BDF80010384600F098F8AC
:10FA00000820E6E70420A0753068A061A4F80A90F9
:10FA100001A8FEF7B7FA46B1C6F804A0E1680648A7
:10FA2000316086F80AA000893081FEF75DFB002076
:10FA3000CFE7000030230020DC2B00202DE9F84325
:10FA40000D46898A374A01EB810102EB810630B10C
:10FA500029463046FDF7E4F90120BDE8F8833189F5
:10FA60007068002400EB81072E48A97DA8384FF06C
:10FA70000E0807294ED2DFE801F00D2D16240440B0
:10FA80004A004460A969016026482749A838FEF762
:10FA9000E9FB30B10220A875042339462A1D0094E1
:10FAA00023E00A20D9E728692A4608B1032000E0AC
:10FAB00001209075042305F10C0207F10801009460
:10FAC00013E00120A8750094E88807F10C01830079
:10FAD0002A690AE028782A4603280CD00620907567
:10FAE000042305F10802391D00941048FBF786FC39
:10FAF000A8B144460FE00520F1E70621A9750A499F
:10FB000040680988FEF72CFC040004D107E041F6A8
:10FB10001D5400E00F2429463046FDF781F92046A8
:10FB20009BE70000B42B002010230020E0230020DE
:10FB300001EB8102034901EB82014A89101AC01EC0
:10FB400048817047B42B002070B5C01C82B240F2CF
:10FB5000FE30824201D3092070BD114B00204FF4CA
:10FB6000806500BF00EB800413F8246096B903EBB6
:10FB700084063489768914443444A4B2AC4209D250
:10FB8000088000EB800003EB800041891144418133
:10FB9000002070BD401C80B20228E3D3072070BD56
:10FBA000B42B00200D0E0F100B0C18190C25002083
:10FBB0002C250020582500200B000300D5810200D1
:10FBC0000C000300D581020018000300D58102005B
:10FBD00019000300D58102000700000000000000AA
:10FBE000000000000000000000000000060000000F
:10FBF0000000000000000000000000000000000005
:10FC000010000000000000000000000000000000E4
:10FC100000000000110000000000000000000000D3
:10FC200000000000000000000100000001000100D1
:10FC300028FC0200010001003CFC02000000000062
:10FC400049DA0200BD950200770A000000000000BA
:10FC5000770A0000000000007ADA000000000000CF
:10FC6000B1D002000700000000000000000000000A
:10FC7000000000000000000049DB0200F9EA020079
:10FC8000D99802003D96020001000000000000002B
:10FC9000010006007C22002085EB0200010000002C
:10FCA0000000000000000000000000000000000054
:10FCB000070000000000000000000000000000003D
:10FCC0000000000003000000000000000000000031
:10FCD000000000000000000005000000000000001F
:10FCE00000000000000000000000000071DE0200C3
:10FCF00050EADA308883B89F604F15F30000C98E50
:10FD00000000005000030050D5C7020031CA0200B5
:10FD100003000000D42900200000000000000000C3
:10FD20000338FDD870470000FC2200200000FFFFD0
:10FD3000DEC0ADDEFF011EF1DEC0ADDEFE011EF154
:10FD40003031323334353637383941424344454611
:10FD50006E72665F6673746F726167655F696E6904
:10FD600074006E72665F6673746F726167655F754B
:10FD70006E696E6974006E72665F6673746F72612D
:10FD800067655F72656164006E72665F6673746F4B
:10FD9000726167655F7772697465006E72665F662F
:10FDA00073746F726167655F6572617365000000EF
:10FDB00040230020001000000400000001000000AB
:10FDC000A19C0200CDF4020051E10200B5F702004F
:10FDD000918C020019E40200B1F70200259F020095
:10FDE00094090300980903000000000000000000CF
:10FDF00000000000000000008C2C0020E0FD02004C
:10FE0000F8FD020004000000556E6B6E6F776E20E7
:10FE10006572726F7220636F6465000000000000FD
:10FE2000C805030001000000740403000200000084
:10FE30006802030003000000E8040300040000005F
:10FE40003C050300050000001C0403000600000040
:10FE5000B8030300070000002405030008000000A9
:10FE60003004030009000000940403000A000000AD
:10FE7000B00503000B000000500203000C0000005E
:10FE8000480403000D000000180603000E000000E7
:10FE9000140503000F0000005005030010000000CF
:10FEA00084050300110000002C060300120000006E
:10FEB00000060300130000009C0503008000000002
:10FEC000D0030300810000000C0303008200000047
:10FED000CC02030083000000AC0203008400000099
:10FEE000E802030085000000F40303008600000020
:10FEF000FC04030090000000980303009100000040
:10FF00008C020300920000005C04030000820000E9
:10FF10006405030001820000B004030002820000B7
:10FF2000CC040300008400002803030001840000C7
:10FF3000D405030002840000700303000384000062
:10FF40004C030300A9B902007DB9020075B9020093
:10FF5000FFFFFFFFFFFFFFFFFFFFFFFFFFFFFFFFB1
:10FF600000000000000000000000D60107010000B2
:10FF7000E0090300E80903000000000000000000A1
:10FF80000100000770FF020080FF0200080000006F
:10FF9000A8FF0200B8FF020008000000B8FF02003E
:10FFA000C8FF020008000000180A0300300A03001E
:10FFB0000000000000000000080A0300180A030007
:10FFC000000000000000000098090300A0090300E1
:10FFD000A0090300C8090300C8090300D8090300E9
:10FFE000D8090300E009030020220020C8FF020016
:10FFF000E8FF020008000000E8090300F809030018
:020000040003F7
:10000000F8090300080A0300F8FF020008000300D3
:100010000800000000404040404040404040414116
:1000200041414140404040404040404040404040CD
:100030004040404040050202020202020202020267
:100040000202020202202020202020202020200264
:1000500002020202020290909090909010101010F4
:100060001010101010101010101010101010101090
:100070000202020202028888888888880808080824
:1000800008080808080808080808080808080808F0
:1000900002020202400000001500030073645F6268
:1000A0006C655F6761705F646174615F6C656E67EA
:1000B00074685F75706461746528292028726571A1
:1000C0007565737429206F6E20636F6E6E6563743F
:1000D000696F6E20307825782072657475726E6550
:1000E000642025732E0000005468652072657175C8
:1000F000657374656420636F6D62696E6174696FA6
:100100006E206F6620545820616E64205258207013
:1001100061636B6574206C656E67746873206973C6
:1001200020746F6F206C6F6E6720627920257520B8
:100130006D6963726F7365636F6E64732E00000088
:1001400054686520626F6F746C6F616465722068BB
:1001500061732077726974652070726F746563745F
:100160006564206974732073657474696E677320A5
:10017000706167652E20546869732070726F6869BA
:10018000626974732073657474696E67207468653E
:10019000207065657220646174612E20546865204A
:1001A000626F6F746C6F61646572206D757374201B
:1001B000626520636F6D70696C656420776974682F
:1001C000204E52465F424C5F53455454494E47536C
:1001D0005F504147455F50524F544543543D302096
:1001E000746F20616C6C6F772073657474696E67CF
:1001F00020746865207065657220646174612E00EA
:10020000616464725F69735F77697468696E5F6265
:100210006F756E647328705F66732C2070616765FC
:100220005F616464722C20286C656E202A20705FE8
:1002300066732D3E705F666C6173685F696E666F92
:100240002D3E65726173655F756E697429290000C2
:100250004E52465F4552524F525F494E56414C49AD
:10026000445F4441544100004E52465F4552524F54
:10027000525F534F46544445564943455F4E4F5491
:100280005F454E41424C4544000000004E52465FDF
:100290004552524F525F464541545552455F4E4F6D
:1002A000545F454E41424C45440000004E52465F6B
:1002B0004552524F525F4D555445585F554E4C4F25
:1002C000434B5F4641494C45440000004E52465F57
:1002D0004552524F525F4D555445585F4C4F434B1A
:1002E0005F4641494C4544004E52465F4552524F8D
:1002F000525F4D555445585F434F4E445F494E49F8
:10030000545F4641494C4544000000004E52465F50
:100310004552524F525F4D555445585F494E4954CE
:100320005F4641494C4544004E52465F4552524F4C
:10033000525F424C455F495053505F52585F504B9B
:10034000545F5452554E4341544544004E52465F0B
:100350004552524F525F424C455F495053505F5097
:100360004545525F52454A4543544544000000000C
:100370004E52465F4552524F525F424C455F495084
:1003800053505F4C494E4B5F444953434F4E4E458B
:1003900043544544000000004E52465F4552524FC0
:1003A000525F4150495F4E4F545F494D504C454D4F
:1003B000454E5445440000004E52465F4552524F50
:1003C000525F4E4F545F535550504F525445440066
:1003D0004E52465F4552524F525F4D4F44554C4529
:1003E0005F4E4F545F494E495449414C495A454428
:1003F000000000004E52465F4552524F525F4D4F33
:1004000044554C455F414C52454144595F494E4922
:100410005449414C495A4544000000004E52465F41
:100420004552524F525F4E4F545F464F554E440017
:100430004E52465F4552524F525F494E56414C49CB
:10044000445F5354415445004E52465F4552524F0B
:10045000525F444154415F53495A45004E52465FF2
:100460004552524F525F494F5F50454E44494E47A7
:10047000000000004E52465F4552524F525F5356A5
:10048000435F48414E444C45525F4D495353494E9A
:10049000470000004E52465F4552524F525F494E50
:1004A00056414C49445F4C454E47544800000000BB
:1004B0004E52465F4552524F525F4452565F545718
:1004C000495F4552525F414E41434B004E52465F99
:1004D0004552524F525F4452565F5457495F4552FE
:1004E000525F444E41434B004E52465F4552524F7D
:1004F000525F494E5445524E414C00004E52465FA9
:100500004552524F525F53544F524147455F4655F3
:100510004C4C00004E52465F4552524F525F4E5572
:100520004C4C00004E52465F4552524F525F494E6E
:1005300056414C49445F504152414D004E52465F36
:100540004552524F525F4E4F5F4D454D00000000E7
:100550004E52465F4552524F525F464F52424944B7
:1005600044454E004E52465F4552524F525F4452F0
:10057000565F5457495F4552525F4F564552525548
:100580004E0000004E52465F4552524F525F494E58
:1005900056414C49445F4144445200004E52465F2C
:1005A0004552524F525F5245534F555243455300A7
:1005B0004E52465F4552524F525F494E56414C494A
:1005C000445F464C414753004E52465F53554343A8
:1005D000455353004E52465F4552524F525F424C74
:1005E000455F495053505F4348414E4E454C5F4133
:1005F0004C52454144595F455849535453000000FB
:100600004E52465F4552524F525F434F4E4E5F43EC
:100610004F554E54000000004E52465F4552524F17
:10062000525F54494D454F55540000004E52465FAD
:100630004552524F525F4255535900007761726ED6
:10064000696E670064656275670000001B5B313B83
:1006500033306D001B5B306D000000001B5B313BD5
:1006600033316D001B5B313B33326D001B5B313B23
:1006700033336D001B5B313B33346D001B5B313B0F
:1006800033356D001B5B313B33366D001B5B313BFB
:1006900033376D00696E666F000000006572726F1F
:1006A0007200000073645F626C655F6366675F730E
:1006B000657428292072657475726E6564202573CF
:1006C000207768656E20617474656D7074696E67FB
:1006D00020746F2073657420424C455F4741545429
:1006E000535F4346475F534552564943455F43482E
:1006F000414E4745442E000073645F626C655F6342
:1007000066675F73657428292072657475726E65FB
:1007100064202573207768656E20617474656D7040
:1007200074696E6720746F2073657420424C455F56
:10073000434F4D4D4F4E5F4346475F56535F5555B0
:1007400049442E0073645F626C655F6366675F7324
:10075000657428292072657475726E65642025732E
:10076000207768656E20617474656D7074696E675A
:1007700020746F2073657420424C455F4741545488
:10078000535F4346475F415454525F5441425F5365
:10079000495A452E0000000073645F626C655F6318
:1007A00066675F73657428292072657475726E655B
:1007B00064202573207768656E20617474656D70A0
:1007C00074696E6720746F2073657420424C455FB6
:1007D000434F4E4E5F4346475F4741502E00000057
:1007E00073645F626C655F6366675F736574282915
:1007F0002072657475726E65642025732077686554
:100800006E20617474656D7074696E6720746F20FA
:1008100073657420424C455F4741505F4346475FD4
:10082000524F4C455F434F554E542E006E72665FDB
:10083000626C655F6761747400000000636C6F63D5
:100840006B000000434C4F434B0000004750494FA2
:1008500054450000505253005541525400000000CE
:10086000554152544500000061746669666F2E6DF3
:100870005F717565756500006E72665F6673746F93
:10088000726167650000000061746669666F2E6DB5
:100890005F6669666F0000007077725F6D676D74E8
:1008A0000000000062616C6C6F632E6C6F675F6D9F
:1008B000656D706F6F6C0000617070006E72665FC6
:1008C000736468006E72665F7364685F626C650073
:1008D0006E72665F7364685F736F6300300A030053
:1008E000202200201402000020650200900A03006C
:1008F00034240020AC2D00000C6A02002C080300F8
:10090000000003033C08030000000000440803004B
:10091000000000004C080300000000005408030021
:1009200000000000580803000000000060080300F9
:1009300000000000680803000000000378080300BE
:100940000000030388080300000000039808030068
:1009500000000000A408030000000003B808030022
:1009600000000303BC08030000000303C4080300E5
:1009700000000303D00803000000030390230020BD
:100980008823002090230020F82C00202024002021
:10099000180000009D6C0200FD7E020000000000B7
:1009A00085AA0200342400204F7302005424002042
:1009B000917D020000000000017E020000000000A6
:1009C000018002000000000007AC02004824002063
:1009D0003D7A02009C280020297D020000000000D2
:1009E00021B3020000000000A1EE020000000000A0
:1009F00059B3020000000000B97302005424002023
:100A00003D7B0200000000007DC2020000000000EB
:100A1000EDC3020000000000398602000000000063
:100A2000DDE402000000000039B302000000000015
:100A3000062BFFFF0A1801042D45DA022A18017956
:100A400009390A01791310240240200A1A184412A5
:100A500020AA4008042544FF02149C06031A3C0403
:100A60001A94041A44041A54041A4C041A5C041A02
:100A700064041A6C041A74041A7C041A84041A8C10
:100A800004515B90D009210B2439936C01240000A0
:02000004000FEB
:10F00000DD850A150100000001000000010000007C
:10F01000000000000000000090AA00002FF19423DF
:10F0200001000000000000000000000000000000DF
:10F0300000000000000000000000000000000000D0
:10F0400000000000000000000000000000000000C0
:0CF05000000000000000000000000000B4
:00000001FF
